:10000000782400203D3200003932000039320000EF
:1000100000000000000000000000000000000000E0
:100020000000000000000000000000003932000065
:1000300000000000000000003932000039320000EA
:10004000393200003932000039320000A9080000BE
:10005000952B00003932000039320000393200009F
:1000600039320000092B0000192B0000292B000059
:10007000392B0000000000000000000039320000B1
:1000800039320000393200003932000039320000C4
:10009000393200000000000000000000393200008A
:1000A00039320000393200003932000039320000A4
:1000B0000000000010B5064C2378002B07D1054B3B
:1000C000002B02D0044800E000BF0123237010BDC4
:1000D0002C02002000000000F8910000084B10B531
:1000E000002B03D00749084800E000BF0748036819
:1000F000002B00D110BD064B002BFBD09847F9E731
:100100000000000030020020F8910000F89100008B
:100110000000000010B50022002302704270002190
:100120004280017103760262C26182600373C0245F
:100130006401C481037443748374C37403752A24F3
:10014000035543758375063C0355C2840285C1750A
:100150002B23C1540133C15410BD0000F0B5D64665
:100160004F464646C0B596B0070016000160CB4A20
:10017000106A80235B02034313620B780520DB07C0
:1001800005D516B01CBC90469946A246F0BD0B782A
:1001900017309B07F5D473783B71002B04D1C04A0C
:1001A000136C04210B4313643B68984633786A460A
:1001B000137069461E20BB4B98471E20BA4B9847C8
:1001C0002C23F25C002A54D0013BF55C337BEB1806
:1001D000DBB2D118C9B28B4221D25219D3B299469F
:1001E000B24B9A4603E00135EDB2A94517D00F2472
:1001F0002C40337BE4185022AD4902A8D047132C81
:10020000F1D8A40002ABE05801A900234B70CB70D9
:100210008B7001330B70C0B2A64B9847E3E7F489AB
:100220005022A34902A8A14B9847132C13D9737DE0
:100230009B00DBB242461370B37DDB01727813433F
:10024000DBB2424653703379342B00D978E19B00FE
:10025000994AD3589F46A40002ABE05801A9002355
:100260004B70CB708B7001330B70C0B2914B9847C1
:10027000DDE7347B50228E4902A88C4B9847132C23
:1002800015D9F48950228A4902A8884B9847132C23
:10029000CDD8A40002ABE05801A900234B70CB706D
:1002A0008B7001330B70C0B2824B9847BFE7A4003C
:1002B00002ABE05801A900234B70CB708B70013367
:1002C0000B70C0B27B4B9847DBE70423102402215C
:1002D0001AE0717C337C102416E0062310240121DF
:1002E00012E00823102400210EE000233024002116
:1002F0000AE000232024002106E00023002400213E
:1003000002E0022310240121090170220A40134354
:1003100042469370F37D17203F2B00D931E7D3700D
:100320003A68537E5BB2002BFBDBF37C728813438D
:100330002422B25CD2001343327D92001343B27C7C
:1003400052001343234342469380337E002B20D038
:10035000102C00D1D6E000D880E0202C00D1B3E0F2
:10036000302C16D1F27C002A0AD0F2698032172094
:10037000FF2A00D905E7326A8032FF2A00D900E758
:100380001720F269FF2A00DDFBE6326AFF2A00DD52
:10039000F7E639684A7E52B2002AFBDB4246137206
:1003A0003A68537E5BB2002BFBDBB38B42469383F0
:1003B0003A68537E5BB2002BFBDB338C42461384DE
:1003C0002C23F35C002B05D0013BDBB217200F2B55
:1003D00000D9D6E62B22B15C17200F2900D9D0E630
:1003E0003868427E52B2002AFBDBF289307B02433E
:1003F000B068024309050A431B04134342461361D4
:100400002A23F35C13750F2393751533F35C002BCC
:1004100012D0F38C294A1720934200D9B1E6424604
:100420009384328D80231B01D31824499BB28B42C5
:1004300000D9A6E64346DA84214B1B685B01E02223
:10044000D20013401F4A516849011268D20E0A4374
:10045000D2B2134342461385002092E6002C98D175
:10046000F27C002A0FD0F269802109018C46624497
:10047000124917208A4200D983E6326A62440F4942
:100480008A4200D97DE60D4A1720F169914200DDCC
:1004900077E6316A914200DD73E67AE700040040B6
:1004A00000080040E130000055300000A533000096
:1004B000B0860000D9310000DC850000FF0F00008D
:1004C0002460800020608000F27C002A0FD0F26956
:1004D000802189008C4662441A4917208A4200D93B
:1004E0004FE6326A624417498A4200D949E6154A02
:1004F0001720F169914200DD43E6316A914200DD47
:100500003FE646E7F27C002A0FD0F269802109021B
:100510008C4662440C4917208A4200D931E6326A7F
:10052000624409498A4200D92BE6074A1720F1693B
:10053000914200DD25E6316A914200DD21E628E79F
:1005400017201EE6FF030000FFFF0000044A137897
:1005500002210B43137053785BB2002BFBDB704717
:100560000018004000B583B0124A936940210B4344
:10057000936101A900230B7005200F4B98470520BC
:100580000E4B98470E4A137801210B431370537892
:100590005BB2002BFBDB0B4B19004031002204C384
:1005A0009942FCD11022084B1A60084B984703B0BF
:1005B00000BDC04600040040E1300000553000009E
:1005C00000180040E002002000E100E04D050000BE
:1005D000002303604360012202724272837202337D
:1005E000C3727047F0B583B005000C0001A9002369
:1005F0004B70CB7023790B70237A8B702078154B5E
:10060000984700201F2D00D8134807222A40920047
:10061000E77AA37A002B01D008231F43EB089B0045
:10062000C31899690F269640B14397403A000A4390
:100630009A61637A002B06D143690122AA40934351
:10064000436103B0F0BD42690123AB4013434361F2
:10065000F7E7C046D9310000001800400368987AD7
:10066000C009704770B5040006680822054B1A607F
:10067000054D2000A8470028FBD1338802221343F0
:10068000338070BD00E100E05D06000070B504003D
:10069000066808218023074AD150074D2000A8474B
:1006A0000028FBD1C123B3713372338802229343F4
:1006B000338070BD00E100E05D06000070B504000D
:1006C0000668074B98470023A382E382054D20006C
:1006D000A8470028FBD1338801221343338070BD23
:1006E0008D0600005D060000F0B583B004000191A6
:1006F00015000668114F2000B8470028FBD1237968
:10070000002B0AD0012B16D11730012D14D8063535
:10071000AD00019BAB5100200EE01720022D0BD83D
:10072000074B019A9A4207D86B469B880C356D009F
:10073000AB53002000E01A2003B0F0BD5D060000BE
:10074000FFFF0000F0B583B00400160001602E4AE0
:10075000936920210B43936101A902230B700420AC
:100760002A4B984704202A4B98472000294B98474A
:10077000B378237133796371274B1C602768338802
:100780003B80B378002B21D01720012B1CD13B8854
:100790009BB23B80F378002B03D03B88802213432D
:1007A0003B801E4D2000A8470028FBD10022B168E5
:1007B00020001B4B984733790020002B04D07B8806
:1007C0008022D20113437B8003B0F0BD3B8804221A
:1007D00013433B80F3781720002BF5D10F4D2000F9
:1007E000A8470028FBD10022B16820000C4B984795
:1007F0000A4D2000A8470028FBD10122F168200003
:10080000074B9847D7E7C04600040040E13000009E
:1008100055300000BD060000200300205D060000EA
:10082000E9060000F8B504000E0003791520002B3E
:1008300000D0F8BD2768034D2000A8470028FBD151
:10084000BE82F6E75D060000022A0BD00379002B7A
:1008500005D0012B12D11633012A0DD802E017233F
:10086000022A09D8931C9B001950838A01219140C8
:100870000B439BB283820023180070471723FBE7CA
:1008800010B5046802290BD001228A4003231340CB
:10089000E371C38A01228A4013439BB2C38210BD15
:1008A0008023E371F5E7000010B5144B1A68146853
:1008B000D18A938A1940207AE379034058B20028FC
:1008C00006DBD8070FD5CB070AD40123237210BD4E
:1008D0004B0702D480232372F9E713699847F9E79D
:1008E00093689847F1E79B07F1D58B0702D4022361
:1008F0002372ECE7D3689847F9E7C046200300204D
:10090000F0B5C64600B50C00904600280FD1002A6D
:1009100011DD8F18094E0A4D306821002B68984769
:100920000134BC42F8D1404604BC9046F0BD0123DE
:100930005B429846F7E78046F5E7C0462C03002067
:1009400024030020F0B5C64600B50E00150001389E
:10095000022810D8002A11D000240C4B98460C4FC6
:1009600043461868315D3B689847002808DB01342E
:10097000A542F5D106E00124644203E0140001E041
:1009800001246442200004BC9046F0BD2C030020EA
:10099000280300200122034B1A608022D200024B60
:1009A000DA617047D80300200044004170B582B07E
:1009B00005000E0000226B46DA80064C6B46991D3E
:1009C0002800A0470028F9D16B4606331B883370F6
:1009D00002B070BDA721000070B505008CB2034EB7
:1009E00021002800B0470028FAD170BD7D21000009
:1009F00010B58CB06846104B984700236A461373B5
:100A0000023353700D4C0E4920000E4B984722685C
:100A1000537E5BB2002BFBDB0F23937513761378A9
:100A200002210B431370054B1A68537E5BB2002BF7
:100A3000FBDB0CB010BDC04615010000A403002074
:100A4000004000425D01000010B584B000236A46FA
:100A5000D37013710293039313809370044C054970
:100A60002000054B98472000044B984704B010BD68
:100A70003803002000140040450700006506000010
:100A800010B5074C022207492000074B9847022166
:100A90002000064B98470022054B1A6010BDC04647
:100AA0003803002095090000490800008108000073
:100AB000D8030020F0B585B0564B1B68002B57D1EA
:100AC000554B00930E236B440F226A4402A903A8DE
:100AD000524CA04705004F4B1B68002B4CD14D4B8F
:100AE0001B68002B54D14E484E4B984700244E4E65
:100AF0004C4F029B195D3000B8470134102CF8D1DF
:100B000020204A4B9847484E464F029B195D3000C3
:100B1000B8470134142CF8D12020444B9847424E5A
:100B2000404F029B195D3000B8470134182CF8D1B2
:100B300020203E4B98473C4E3A4F029B195D3000B7
:100B4000B84701341C2CF8D1029B197F3848354B2B
:100B50009847029800233749C25CCA5401331C2BC2
:100B6000FAD12C4B1B68002B18D1002005B0F0BD2A
:100B70003148324B9847A3E70E236B441B780F2272
:100B80006A44127803A909882D48264CA047A6E795
:100B900003AB19882B48234B9847A4E7254EB3682D
:100BA00072683168F068009027481E4CA047274BB8
:100BB00032691A6011002648A04772691100254861
:100BC000A047254FB069B84702000B002348A04753
:100BD000114B1868224B9847FC218905214B9847F7
:100BE0002149224B9847B84702000B002048A047F4
:100BF00029002048A047029B197F1F48A0471C21BD
:100C000002981E4B984701001D48A0471D480B4BFA
:100C10009847AAE7AC030020CC030020C91C0000C1
:100C2000E4880000A93C0000EC880000DD3C0000E6
:100C3000F4880000E40300206C880000C53D00003B
:100C40009C880000CC880000FC8800000C0000207C
:100C50002089000048890000E58400006C890000BC
:100C6000096900009163000000000643D16500009F
:100C700090890000A4890000B48900005516000086
:100C8000D4890000F489000030B583B0204B1900EE
:100C90001C3100221A7001338B42FBD11D4A1E4BBE
:100CA0001A601E4A1E4B1A601E4A1F4B1A60184CCF
:100CB0001E4B1A6822605A686260DB68A3601C4B96
:100CC0001D6865611B4B1B6823611B4B18681B4B20
:100CD0009847FC2189051A4B98471A491A4B98479F
:100CE000A0611A4B1B68002B08D1094C1C21200065
:100CF000174B984720771D2003B030BD154B984700
:100D0000009001912A0029001348144B9847ECE702
:100D1000E40300209A99993F300300200000AA4381
:100D2000500300203333B34000040020B8030020F8
:100D3000100000200C000020CC03002009690000F6
:100D40009163000000000643D1650000AC03002061
:100D500055160000E584000028880000A93C00002A
:100D6000F0B583B0334B1B68002B55D1324B9847FD
:100D7000324B186000284CD02E4B1B68002B4FD1F3
:100D80002F48304B9847304C270010372F4E2D4DB1
:100D900021783000A8470134A742F9D120202C4BFC
:100DA00098471024284F294E264D395D3000A8471A
:100DB0000134142CF9D12020254B9847224F234E83
:100DC000204D395D3000A8470134182CF9D120207E
:100DD0001F4B98471C4F1D4E1A4D395D3000A847D8
:100DE00001341C2CF9D1184C217F1A48154B984717
:100DF000124B1878012301933B3300930023032205
:100E00002100154CA0470B4B1B68002B0DD1134B39
:100E10009847012003B0F0BD1148124B9847A5E751
:100E200001001148074B9847AAE710480D4B984717
:100E3000EDE7C046AC030020890C0000D40300207D
:100E4000688A0000A93C0000E4030020EC88000050
:100E5000DD3C0000F4880000491A0000D5170000AE
:100E6000248A0000C53D0000548A0000288A000042
:100E700010B50848084CA0470848A0470848A047B4
:100E80000848A0470848A0470848A0470848A04786
:100E900010BDC0469C8B0000C53D0000B08B00001B
:100EA000C88B0000E48B0000108C0000308C000028
:100EB000508C000070B5464B1868437E5BB2002B27
:100EC000FBDB03691F2293430361437E5BB2002B6C
:100ED000FBDB437E5BB2002BFBDB037B0222134375
:100EE0000373437E5BB2002BFBDB0121042502244C
:100EF00001E011420AD1037EDBB20A001A401D4212
:100F000000D022431C42F4D02A43F2E7437E5BB276
:100F1000002BFBDB418B89B201230376027ED2B228
:100F20001340540701D502242343920701D504221C
:100F300013435B0701D5022303762648264B9847C7
:100F4000234B1868437E5BB2002BFBDB03691F2237
:100F500093431E3A13430361437E5BB2002BFBDBDA
:100F6000437E5BB2002BFBDB037B02221343037344
:100F7000437E5BB2002BFBDB01210425022401E050
:100F800011420AD1037EDBB20A001A401D4200D092
:100F900022431C42F4D02A43F2E7437E5BB2002B8B
:100FA000FBDB418B89B201230376027ED2B2134070
:100FB000540701D502242343920701D50422134389
:100FC0005B0701D5022303760448034B984770BDA5
:100FD000A40300206C8C0000A93C0000788C000069
:100FE000F0B5D6464F464646C0B594B00026B84B3D
:100FF0001E600027B74B1E70B74B9847B74B9847FA
:1010000003AB8022D20503925E60FF221A819E729A
:10101000DE72FE3A24215A5401315A5425329E542C
:1010200001329E549E6205329E5401329E545E618E
:101030001E820022DA761F761F775F7613229A7659
:101040005F77E12252021A6280225203DA60A44AD8
:101050001A63A44A5A63012252429A63DA63A24F86
:10106000A24E03AAA2493800B0470028F9D19E4EEB
:10107000A04B1E60A04AA14B1A60A14AA14B1A6066
:1010800003AA9B493000994B98479F4B98461B6891
:10109000986800219D4FB84743461B685868002157
:1010A000B8473368DA69002AFCD11A6802210A437A
:1010B0001A60974B9847974B9847974B19889748D2
:1010C000974B984703AE012373700022B2703370C0
:1010D00031000A20934B98469847934F8023DB00BA
:1010E000BB6131000820C04780235B00BB61310039
:1010F0000920C04780239B00BB618C488C4EB047C1
:101100008C4A8D498D48B0471C218D48B04700203E
:101110008C4B98478C4B1B7ADBB20100D9408B4833
:10112000B0478B4B98478B4B19001C3100221A702B
:1011300001338B42FBD14023013B002BFCD14022E9
:10114000854B1A60854B1B681968854E3160854B4D
:101150001868021D1A6002687260070008371F6075
:101160004368B3608068F060594E3668002E03D043
:1011700000907D486E4EB0477C4B98470020714BE5
:101180009847020000237A48002180185941794A83
:101190000023794EB047794B9847794B98474C4B91
:1011A0001B68002B02D07748774B9847774EB146A3
:1011B0001DE000234A461360754B98470020614BA1
:1011C0009847040000256A48002100196941694ACE
:1011D0000023694FB847694B98476E4B984709E021
:1011E0004E21694440486C4B984700280AD0336828
:1011F000002BDED1694B1B68002BF1D00022674B1E
:101200001A60EDE74E236B441A881300303B99B205
:1012100049294FD88B006249CB589F464C4B984781
:10122000E5E7414B80225200DA611969C905C90F0F
:101230005C483F4B98475C4B9847D8E73A4B802235
:101240009200DA6119698905C90F5848384B9847E7
:10125000554B9847CBE71E4B1B68002B08D101224A
:101260001B4B1A601A4B19685148314B9847BEE71F
:101270000022174B1A60F5E7164B1B78002B08D19C
:101280000122144B1A70134B19784A48284B98477F
:10129000ADE700220F4B1A70F5E7302A14D0303A30
:1012A000FA23DB005A43444B1A60434B1968434806
:1012B0001F4B98474E276F44414B9A4639880A483E
:1012C000D0470028FAD192E73E4A3B4B1A60ECE740
:1012D000AC030020580200200D320000F10900008C
:1012E000020016000200170048020020811E0000C4
:1012F000001400422C030020D9090000280300201C
:10130000AD090000240300205C000020D93D00004E
:10131000490A0000810A00001C0000203803002058
:1013200025080000E92B000000440041708A0000FD
:10133000A93C00008C8A0000988A0000A48A000062
:10134000C08A0000C92F000000040040E48A0000A9
:10135000710E0000E4030020C803002014000020E8
:10136000B803002018000020F48A0000C515000012
:10137000571B0000581B00007D6100000100002089
:10138000D5170000188B0000F51900001404002088
:10139000B50A0000610D0000A7210000D80300205D
:1013A000008700002C8B0000B50E0000408B000071
:1013B000548B0000688B0000100000207C8B000024
:1013C0007D210000204E00000122014B1A70704761
:1013D0009D0200200122014B1A6070471404002076
:1013E00010B5064C022206492000064B98473722CA
:1013F000A35C04210B43A35410BDC0461C04002071
:10140000C913000019250000F0B591B02A4C05233E
:10141000237000236370A37001A901224A708B70AE
:101420000A700520254B98472378D9090022002906
:1014300004D15A09D20122498C4662441F26334006
:10144000012529009940916102AC25700023039386
:10145000049323746374A574E57423752422A35440
:10146000183A002108A8174B9847174BA36180230F
:101470005B02E360154BA36201235B42E362144B02
:101480002363144B6363144F220014493800144B38
:1014900098473C682000134B98470640B540124BD4
:1014A0001D603A68D369002BFCD1236802221343E4
:1014B000236011B0F0BDC04658040020E92B0000A5
:1014C00000440041B7330000A0860100030004007F
:1014D00003000600030007001C040020000800426F
:1014E00011220000E52A000000E100E010B584B000
:1014F00001AC2000074B98470E2301930023636043
:1015000023720233E37221000E20034B984704B08C
:1015100010BDC046D1050000E505000010B5002251
:101520000E210448044B984700210E20034B984796
:1015300010BDC046D5130000492B0000752B0000DC
:1015400010B5164B802212025A615A615A615A61D3
:101550009A619A619A619A61802212055A6100200B
:101560000F4B98470200002392185B410D48002161
:10157000801859410C4A00230C4CA0470C4B98474B
:101580000C4B1B78002B04D101220B4B1A6000205E
:1015900010BD0A480A4B9847F6E7C0460044004190
:1015A000C92F0000571B0000581B00007D61000080
:1015B000010000205802002054020020A08C0000EE
:1015C000C53D0000F0B583B0174B9847174B9847BF
:1015D0000125174B1D70BFF35F8F62B601AC6570BC
:1015E0000023A3702570134F80231B05BB612100CE
:1015F0001B20114EB047257080231B02BB612100C8
:101600000F20B0470D4B98470D4B98470D4B1B785B
:10161000002B04D10C4B9847002003B0F0BD0B48C1
:101620000B4B9847F6E7C046ED1400001D1500006F
:101630005B00002000440041E92B00000914000079
:10164000E113000058020020411500008C8C0000BE
:10165000C53D0000002909D00300411800201A7878
:10166000801AC0B201338B42F9D170470020FCE7E9
:10167000F0B5CE46474680B585B001900291039201
:10168000444C012244492000444B98470020444BDD
:1016900098470300180000211A000B0012184B4154
:1016A00012184B41150F190129431001801A994155
:1016B0003C4A0023801859413B4A00233B4DA84730
:1016C0003B4B98476B469B89029A01992000394C05
:1016D000A047394B1870002821D1384C384B994617
:1016E0002F4B98464B461B78002B21D10020C0473A
:1016F000060000272B480021801979412A4A00233F
:101700002A4DA8472A4B9847013C002CEAD10022D9
:1017100021492048214B98471220404221E00022D5
:101720001D491C481D4B9847234B1878404218E030
:101730000022234B1A70019B1B78224AD45C002C98
:1017400014D1002214491348144B984702990B787E
:101750001D4A1370497851707F2293431B4A1370BE
:10176000039805B00CBC90469946F0BD00200C4B88
:1017700098470200002320000021154CA047094A89
:10178000002380185941084A0023084CA047084B01
:101790009847D6E71C0400205804002025240000A8
:1017A000C92F0000BFCF6A00C0CF6A007D61000072
:1017B00001000020312500005B040020B90B00006F
:1017C0009D020020200000200804002010040020BA
:1017D000BD61000000B583B001A8054B1A880280E6
:1017E0009B78837003226946024B984703B000BD83
:1017F000848C00007116000000B583B001A8054B71
:101800009A8802809B79837003226946024B98472D
:1018100003B000BD848C00007116000010B582B0CA
:10182000040001A801230370002343708370032286
:101830006946034B98476B469B78237002B010BDF6
:101840007116000010B582B0040001A803230370D4
:1018500000234370837003226946034B98476B460D
:101860009B78237002B010BD7116000000B583B0E4
:10187000010001A804220270002242708270C2702E
:101880000432024B984703B000BDC04671160000F9
:1018900070B58AB004000E0001AD2322002128009B
:1018A000064B984705232B706C700334E2B231006D
:1018B0002800034B98470AB070BDC046B7330000FC
:1018C0007116000070B58AB004000E0001AD23222D
:1018D00000212800064B984706232B706C700334B8
:1018E000E2B231002800034B98470AB070BDC046F1
:1018F000B733000071160000F0B58DB005000E0082
:101900001700019303AC232200212000074B9847C6
:10191000082323706570A670E7700535EAB2019957
:101920002000034B98470DB0F0BDC046B733000010
:101930007116000070B592B005000C0009AE2322AC
:10194000002130000D4B98470B2333707570002D2C
:101950000CD0230026226A44691EC9B201316118E5
:1019600018781070013301328B42F9D10235EAB296
:10197000694609A8024B984712B070BDB733000002
:101980007116000070B592B005000C0009AE23225C
:10199000002130000D4B98470C2333707570002DDB
:1019A0000CD0230026226A44691EC9B20131611895
:1019B00018781070013301328B42F9D10235EAB246
:1019C000694609A8024B984712B070BDB7330000B2
:1019D0007116000000B583B001AB0D221A7058706B
:1019E00099700A3A69461800014B984703B000BD48
:1019F0007116000030B585B004000D4B1B78002B2C
:101A000008D10C4A5378127801000B480B4CA047C0
:101A100005B030BD6B46002203210120084DA847C8
:101A20006B465A7921000748044B9847F0E7C046B7
:101A30001004002008040020D88C0000A93C0000FD
:101A4000F9180000B88C0000F0B583B00090019147
:101A50007E4B984700207E4B98474622002300216A
:101A60007C4EB0477C4A0023801859417B4A0023B2
:101A70007B4EB0477B4B98477B4B1B78002B00D0AD
:101A80008FE07A487A4B98470500774B1B78002BFC
:101A900000D08AE0774B1B78774AD15C2120774BC6
:101AA0009847714B1B78002B00D091E074490920B6
:101AB000744B98476C4B1B78002B00D08CE00020B7
:101AC000634B9847642200230021624EB047624A6C
:101AD000002380185941614A0023614EB047614B91
:101AE000984701990098684B98475F4B1B78002BEB
:101AF00000D075E00022654B1A601A001368002BB5
:101B0000FCD00022614B1A600026514F01360020A4
:101B1000B8475F4A002300214E4CA0474E4A00239D
:101B2000801859414D4A00234D4CA0474D4B9847D2
:101B30004E4C20004E4B98476378DB0601D4282E8C
:101B4000E4D1494B1B78002B56D10020404B9847DD
:101B50004622002300213F4CA0473F4A0023801823
:101B600059413E4A00233E4CA0473E4B9847374BD5
:101B700098473D4B1B78002B64D10020344B98478D
:101B8000462200230021334CA047334A002380180B
:101B90005941324A0023324CA047324B984703B098
:101BA000F0BD3C483C4B98476BE73C483C4B984762
:101BB000002D09D02D4E75193A4F394C3178380027
:101BC000A0470136AE42F9D13748384B984761E714
:101BD0003748314B984769E736482F4B98476EE7AF
:101BE00035482D4B9847204B1B78002B00D181E7BF
:101BF00032482E4B98477DE77200921931003048E9
:101C0000274CA0471B4B1B781B4AD35C9A06920FAC
:101C1000072119402B48A0471448154B9847050049
:101C20001E48A047002D09D0104C65191D4E1C4FB1
:101C300021783000B8470134AC42F9D11A481B4B27
:101C4000984782E71348144B984796E7F917000026
:101C5000C92F0000BD610000BFCF6A00C0CF6A007D
:101C60007D61000001000020580200205C0200207D
:101C70006D1800009C0200204C000020D5190000C7
:101C800040000020851900003519000014040020D0
:101C9000B80B00001C8D0000F5190000308D00000D
:101CA000A93C0000488D0000B48C0000C53D000038
:101CB000508D00006C8D0000848D0000988D000018
:101CC000A88D0000D08D0000F0B5D6464F464646A0
:101CD000C0B582B00500894690469A46504B19001F
:101CE000403100221A7001338B42FBD14D4F4E4ED2
:101CF0000020B847FA22520000230021B0474B4A87
:101D00000023801859414A4A00234A4CA0474A4BB5
:101D10009847434C2000494B98476378DB06E7D54A
:101D20003F4FFE7800203F4B9847454A0023002153
:101D30003D4CA0473D4A0023801859413C4A0023AE
:101D40003C4CA0473C4B984738003E4B98473C786A
:101D5000200002230193002C27D10A9B1860304CED
:101D60002000394B984724782C80651E1F2D2FD9D1
:101D7000364B1B78002B3DD1354B9847334B1B78A6
:101D8000002B48D1072333404246137003231E40E3
:101D900053461E70224B03334A461360019802B02B
:101DA0001CBC90469946A246F0BD1D4F3900294BF8
:101DB0009847FB1CE11C791800201A788018013321
:101DC0008B42FAD12100244B984700230193C4E7AA
:101DD000134F39002000214B9847F81C2900204B55
:101DE00098473B199B788342C2D00123019A1A433A
:101DF0000192BDE71B481C4B9847094DEC1C23354D
:101E00001A4F21781A48B8470134A542F9D1194828
:101E1000154B9847B0E71848184B9847B2E7C046AB
:101E20005C020020C92F0000BD610000BFCF6A0026
:101E3000C0CF6A007D610000010000206D18000025
:101E400088130000451800001D18000058020020EB
:101E5000F917000091180000155E0000C518000079
:101E600055160000F08C0000C53D0000A93C0000A4
:101E7000108D0000B48C00001C8D0000F5190000CE
:101E8000F0B5DE4657464E464546E0B591B00500F2
:101E90000C00160029600800AD4B9847020023682B
:101EA0000520DB0706D511B03CBC90469946A246FA
:101EB000AB46F0BD236817309B07F4D4A549086AE8
:101EC000971C0123BB4003430B620FA92D27F35D31
:101ED0000B701432D3B2029318009F4B98470298AC
:101EE0009E4B9847F05D00219D4B9847F37A6B71AC
:101EF0002423F35CAB712523F35CEB71F37E2B722F
:101F0000337F6B722B6898461800914B98471430BA
:101F100000220E2306A98C4663441A80328A02925C
:101F20008023DB019A4200D19FE00FD9C023DB015F
:101F3000029A9A4200D193E080231B029A4200D079
:101F400001E1032306930023079308E080239B010C
:101F50009A4200D0F7E0102306930F3B07933368B3
:101F60009B46F368049373699A46337E0593262350
:101F7000F35C039373689946002B00D1A1E08023A2
:101F80005B05994500D185E0737E002B02D0B37EBE
:101F9000424693732A68029FD369002BFCD10E330B
:101FA00006AA944663441B88424693815B46049A82
:101FB0001343524613434A4613431F43059B1B02D8
:101FC0001F43039B5B071F432723F35C002B01D1B7
:101FD00004331F43737E9B02327F52021343727F8E
:101FE000120213432422B25C520413432522B25C32
:101FF00012041343B17AF27A114319433389FF2B48
:1020000000D182E080225204174319432C23F35C51
:10201000002B03D1534B9B789B0701D580231F4393
:102020002A68D369002BFCD1434659602A68D369DA
:10203000002BFCD143461F600EAB80221A70002299
:102040005A70DA709A70336B0A93736B0B93B36B9D
:102050000C93F36B02930D9300270AAD424E63E09D
:1020600008230693073B079379E733689B46F36899
:10207000049373699A46337E05932623F35C039396
:1020800073689946002B18D080235B05994501D0D1
:10209000002025E02723F35C002B00D074E7336A8F
:1020A0001F00C0B2314B984701000E2206AB9C4680
:1020B000624438002E4B984712E008230693002311
:1020C00007932723F35C002B0ED0069B0093079BFE
:1020D0000E2206A98C466244B16A306A254FB84781
:1020E000002800D0DFE64FE7336A1F00C0B21F4B65
:1020F00098470100069B0093079B0E2206A8844682
:10210000624438001B4FB847EAE7F37E002B00D14A
:102110007CE78023DB041F4378E72000164B9847B9
:1021200007E00137042F0CD0F9B2BB005859002842
:10213000F3D0431CF5D00EA90870000CC0B2B04714
:10214000EFE70020AFE6102306930023079306E78E
:10215000592A000000040040E13000005530000022
:102160001129000000200041D9310000FD3000009D
:10217000532800007D2800005D290000C3791C223F
:10218000002B01D1100070470368187E173AC00772
:10219000F8D5DA69002AFCD1198502211A7E0A4293
:1021A000FCD00022EEE782791C23002A01D118001E
:1021B00070470268107E173B4007F8D5D369002BA3
:1021C000FCD1538BDBB298061DD0980703D50223B0
:1021D00053831833EBE7580703D5042353831A338B
:1021E000E5E7D80703D5012353831233DFE7D80689
:1021F00003D5102353833233D9E79B0603D520231D
:1022000053832133D3E7138D0B800023CFE70000E6
:10221000F0B58BB005000C00160029600B681C207F
:102220009B0701D50BB0F0BD0B681738DB07F9D45D
:1022300008006F4B98476F4A116A871C0123BB4007
:102240000B43136209A92427F35D0B701430C3B24A
:1022500001931800684B98470198684B9847F05DC8
:102260000021674B98473378012B3FD03378002B00
:1022700003D123680822134323602B000C33290069
:102280002831002204C38B42FCD10023EB62AB62F5
:102290000024AB862B863633EC540133EC540133E7
:1022A000EC54353B6B722C712868514B98470700F2
:1022B0005449554B9847BF00544BFD502F6804AB11
:1022C00080221A705C707F3A9A70DC703378002B31
:1022D00002D1002204AB9A70B36A0593F36A0693A5
:1022E000336B0793736B089300240BE023680C2275
:1022F00013432360BAE73800454B98470AE001349E
:10230000042C10D0E1B2A30002AA0C201218D0585D
:102310000028F0D0431CF2D004A90870000CC0B211
:102320003C4B9847EBE733786B71337CAB71B37CF4
:10233000EB71337D2B72002202ABDA803378012BF4
:1023400012D03378002B26D1B069B28B7B6AF17F33
:102350000904B47F2143194379622023F35C002BE5
:102360001BD040231A4318E02868214B98471430AB
:10237000C0B2294B9847010002AB9A1DB069274BA8
:10238000984703001720002B00D04BE702AB063321
:102390001B783B73D5E7002200207368B1680B43BC
:1023A000F1680B430343317C0A43717C002903D15C
:1023B0001B498978890701D580210B43B17C00290D
:1023C00002D0802189020A43F17C002902D08021B9
:1023D00089000A43317D002902D0802189010A4306
:1023E00039680B433B607B681A437A60002019E729
:1023F000592A000000040040E13000005530000080
:102400001129000075250000A52A000060040020A5
:102410005D290000D9310000FD3000005328000084
:102420000020004110B544791523012C01D018007B
:1024300010BD047A0023002CF9D1002A58D04B7823
:10244000002B44D003681B7EDB0710D40A78D10927
:102450000023002904D15309DB012E498C46634433
:102460001F21114001228A409A610523DFE70A7883
:10247000D4090023002C04D15309DB01254CA446C8
:1024800063441F2414400122A2405A6103681A7E4B
:10249000D20701D58A789A62C2790023002AC6D170
:1024A00002680421137E0B42FCD0117E00234907F1
:1024B000BDD5538B5B0701D5042353838379012B4F
:1024C00002D0936A0023B2E7936A0023AFE70A7849
:1024D000D1090023002904D15309DB010D498C46A1
:1024E00063441F21114001228A405A6100239EE764
:1024F0000A78D1090023002904D15309DB010549D9
:102500008C4663441F21114001228A409A610023B6
:102510008DE7C04600440041931C9B00C3185960DE
:102520003621012393401A00435C13434354704700
:1025300030B51724002B01D1200030BDC5790534FA
:10254000002DF9D01C34055D333C052DF4D0838675
:1025500003868262C16205223823C254363B43722D
:1025600003689A7542790024002AE5D102321A766E
:102570009A75E1E7F8B58000854BC4582668372383
:10258000E35C3622A75C1F40337EB57D1D40EB0720
:102590002ED56379012B25D0002B29D1637A002B0E
:1025A00026D02168E26A1378DBB2501CE062A07981
:1025B000012800D169E09BB2DB05DB0D8B62A38EA5
:1025C000013B9BB2A386A38E9BB2002B10D101339B
:1025D0003375637A012B0BD1E379002B08D10233D9
:1025E000B37505E0637A002B3ED0637A002BD8D117
:1025F0006B0711D5738B5B0751D5637A012B08D01C
:102600001E223823E254353B6372023333753B0795
:1026100041D4B36A04237383AB0715D56379002BC8
:102620000ED107333375053B3376013363720023D4
:10263000A386238638330022E254FB0600D57FE0D0
:102640006379012B00D17FE02B0708D56379002B3C
:1026500005D1083333753376BB0600D58AE06DB2F9
:10266000002D00DA8AE0F8BD4A4B1B88B362638E06
:10267000013B9BB26386638E9BB2002B01D1013379
:1026800033756379012BB0D086E75078000203439D
:102690000232E26290E72000A3699847B9E7637AC3
:1026A000012B27D023689B6ADB05DB0DDAB2A16A18
:1026B0000A70A26A511CA162A179012933D0238E2C
:1026C000013B9BB22386238E9BB2002BA4D1002218
:1026D0003833E254343B3375637A022B29D0637A62
:1026E000002B00D098E7BB0700D495E720002369B2
:1026F000984791E723689B6A638E013B9BB2638690
:10270000638E9BB2002B00D086E704333375002222
:102710003433E254353B6372FB0700D47CE720007E
:10272000E368984778E71B0A5370A36A0133A362F2
:10273000C5E77B0700D46FE72000636998476BE724
:102740002000E36998477BE7637A012B00D086E796
:10275000E379002B00D082E70233337501336372D3
:1027600000223533E254FB0700D46DE72000E36814
:10277000984769E72000236A984770E780233375FC
:1027800033767B0600D46EE7636A200098476AE7D9
:10279000600400205C040020F0B5DE4657464E463B
:1027A0004546E0B587B08046049116001F00002220
:1027B000002300218B463F24012021000096019731
:1027C0005C4603944446059413E02024641A0500F3
:1027D000E540A84614E0009C019D121BAB415C46FD
:1027E0004D462C43A346039C45462C430394013994
:1027F00025D3202464420C19E7D40500A540A8463F
:1028000004008C40A14692185B4114001D00059EF7
:102810004F463E40B446049E47463E40B24666465A
:1028200057463E4303D00600264332002B00009C4F
:10283000019D9D42DBD8CED19442D8D8CBE7039BF3
:102840005846190007B03CBC90469946A246AB4694
:10285000F0BD10B5490840230024814202D218007F
:1028600010BD1C00091A631C9BB28842F9D9402391
:10287000FF2CF4D814800023F1E70000F0B583B0FA
:102880000F00160008AA117804004C434022BC42F5
:1028900002D9100003B0F0BD002B14D102000800D3
:1028A0000021194CA04701003A0000230020174CDA
:1028B000A04700220123121A8B41120C1B041A4359
:1028C00032800022E5E70022012BF9D10A00002323
:1028D00000210D4CA04702000B000092019338002C
:1028E00000210A4CA047050080239B01402298420A
:1028F000CFD8790FF800009A019BA047EA00821A0E
:10290000D2B252032A43DBE7BD61000099270000E1
:1029100010B582B004000E4B1B78002B07D00029A5
:1029200005D10B4B5B78834210D01D200CE001A930
:102930000C701320074B98471320074B9847044B04
:102940005C7001221A70002002B010BD0020FBE76D
:10295000A0020020E1300000553000002B4B9842CF
:1029600023D00FD92A4B98422FD02A4B984242D1DC
:1029700001293AD0002946D0022938D0032938D07D
:10298000002039E0244B984235D1012907D0002995
:1029900033D0022905D0032905D000202CE01F48A0
:1029A0002AE01F4828E01F4826E0012907D0002917
:1029B00025D0022905D0032905D000201CE01A48A3
:1029C0001AE01A4818E01A4816E0012907D0002931
:1029D00017D0022905D0032905D000200CE01548A6
:1029E0000AE0154808E0154806E0154804E01548D7
:1029F00002E0154800E0002070471448FCE703207F
:102A0000FAE71348F8E71348F6E7C046000C00421F
:102A100000100042001400420008004203000500BC
:102A200003000600030007000300010003001E006E
:102A300003001F000300090003000A0003000B004D
:102A40000300110003001200030013000300040040
:102A5000030008000300100030B585B06A460F4B34
:102A600032CB32C21B6813600300009A824211D03D
:102A7000019A82420AD0029A824209D00020039A27
:102A80009A4201D005B030BD033004E0012002E0DD
:102A9000022000E00020C0B2F4E7C046F88D00003C
:102AA0007047000030B50B4B1B78002B0ED10A4C41
:102AB0000A4D25600A4B00221A6065605A60A560C5
:102AC0009A60E560DA600132024B1A708000024BB6
:102AD000C15030BDA2020020A4020020A12A0000A3
:102AE0006004002010B582B001AC092323700133CB
:102AF00063700133A3700133E370024B9847205693
:102B000002B010BD592A000010B5024B1B6800200E
:102B1000984710BDA402002010B5024B5B6801204D
:102B2000984710BDA402002010B5024B9B680220FC
:102B3000984710BDA402002010B5024BDB680320AB
:102B4000984710BDA40200201723002A01D01800C6
:102B500070478B00064A9B58002B03D0834205D058
:102B60001D23F4E7890088500023F0E70023EEE7F7
:102B7000E00200201723002901D01800704700222E
:102B80001F2800D8024A01238340D3600023F4E7C2
:102B90000018004070B50022104B1A700023104935
:102BA0001F25104E0D4C0AE00D4908E02378013333
:102BB000DBB223700F2B10D800211F2BF4D9280073
:102BC00018400122824008691042EFD00A619B0040
:102BD0009B59002BEAD09847E8E770BD70040020AD
:102BE00000180040E002002000B583B001AB802255
:102BF0001A700A785A704A789A708A78DA701900CE
:102C0000014B984703B000BDD93100007047000068
:102C10000C4B1B68002B06D1EFF31083002B07D061
:102C20000022094B1A70074A13680133136070477A
:102C300072B6BFF35F8F0022044B1A700132024B51
:102C40001A70F0E7B4020020B80200205B000020F8
:102C5000084B1A68013A1A601B68002B09D1064B11
:102C60001B78002B05D00122044B1A70BFF35F8F35
:102C700062B67047B4020020B80200205B0000205A
:102C800010B5082803D880001B4B1B589F46002016
:102C900030E01A4B18692DE0194B1B6A9B059B0FFE
:102CA0001848D84026E0154B586923E0134B1B68A1
:102CB00000209B071ED512491022CB681A42FCD077
:102CC0000E4B1B685B0701D40F4813E000200F4B2D
:102CD00098470A4B9B681B041B0C58430AE050237F
:102CE000074AD35C00205B0704D5044BD86801E099
:102CF0008020000210BDC046088E0000BC020020EB
:102D00000008004000127A00006CDC02FD30000078
:102D100070B50C490B6A0478857840780122104020
:102D200080014026B34303432A40D20180208343DD
:102D300013430322224012020348034013430B6251
:102D400070BDC04600080040FFFCFFFF082803D804
:102D50008000254B1B589F46172044E0234A136AE6
:102D600002210B43136200203DE0204A93690221B7
:102D70000B439361002036E01C4A138A02210B4367
:102D8000138200202FE0194A938A02210B43938279
:102D9000002028E016490B68022213430B60134BF6
:102DA0009A8419000E32CB681A42FCD0104A9168FE
:102DB0000E4BD96252689A6200229A84190010322E
:102DC000CB681A42FCD00A4B1B689BB2074A93841B
:102DD000002008E0054944228B5C022003438B5409
:102DE000002000E0002070472C8E0000000800400A
:102DF000BC020020F0B585B0C222D200214B9A60FF
:102E0000214A53681E218B43536001236A46137085
:102E100000241E4DE0B26946A8470134252CF9D1A3
:102E200003A800244470012787700470184B98474A
:102E30000620184B9847184B98476B465C701C72DD
:102E40005C7204236A4613701C33019369460220A6
:102E5000124EB0470220124DA847124B1C725C72F2
:102E60009C72DC7201976B465C7006236A46137095
:102E70001472547269460020B0470020A84705B07C
:102E8000F0BDC0460008004000400041E1300000B5
:102E9000112D00004D2D0000A92E0000CD2E0000A8
:102EA000852F000000040040064A936908210B4367
:102EB00093610122044B1A7019000B781342FCD164
:102EC0007047C04600040040000C004070B506008A
:102ED00004000D782D0205434B78002B02D080238F
:102EE000DB021D434B7A002B02D080231B031D43C2
:102EF0004868012810D9431E184234D1022830D91D
:102F00000223002201325B009842FBD812023243B6
:102F1000140080235B031D430B7A002B02D0802317
:102F20009B031D43134A53785BB2002BFBDB124B10
:102F30009847124B1E700F4A53785BB2002BFBDB95
:102F40000C4B9C601A0053785BB2002BFBDB094AE8
:102F50005368802149020B401D435560084B984738
:102F600070BD0022D2E70402344380239B021D433C
:102F7000D2E7C046000C0040112C0000080C0040B5
:102F8000512C000010B504000B4A53785BB2002BA3
:102F9000FBDB0A4B98470A4B1C70074A53785BB21D
:102FA000002BFBDB044A516880235B020B43536018
:102FB000044B984710BDC046000C0040112C000087
:102FC000040C0040512C000070B504001A4A5378DC
:102FD0005BB2002BFBDB194B9847194B1C70164A50
:102FE00053785BB2002BFBDB134E7068C004C00E3D
:102FF000144B98470500124B1C707668F602F60FCA
:10300000114B1C700C4A53785BB2002BFBDB0A4B54
:103010009C682402240C0D4B9847002E07D1012CEC
:1030200007D9210028000A4B9847050001E0013428
:10303000E540280070BDC046000C0040112C000087
:10304000040C0040812C0000080C0040512C0000B2
:10305000155E000010B50400064B9847064B1C7027
:10306000064A53888021C9010B435380044B98477B
:1030700010BDC046112C0000020C0040000C0040A6
:10308000512C000010B504000F4B98470F4B1C70DB
:103090000F4A53881B05180F53880E490B40538065
:1030A00053880D490B40538011008022D2014B8878
:1030B0001342FCD106494A880302064802401343E2
:1030C0004B80064B984710BD112C0000020C0040AD
:1030D000000C0040FFF0FFFFFFBFFFFF512C00007E
:1030E00010B50C7824020443024B9847A4B2024B5B
:1030F0005C8010BD85300000000C004010B504005D
:10310000064B9847064B1C70064B5C882405240F21
:10311000054B98472000054B984710BD112C000027
:10312000020C0040000C0040512C0000C92F000090
:1031300030B5D378002B35D11378802B29D01B06DE
:1031400080246402234354780225AC4306D194784A
:10315000002C20D18024A402234341605478013CF8
:10316000012C1CD90D042D0CA024E4052C431C4378
:1031700084620D0CD02424062C431C438462D47832
:10318000002C22D15B031CD59378012B1ED041610A
:1031900017E00023D7E7C024E4022343DDE70D4C0A
:1031A0002340DFE741600C04240CA023DB0523430C
:1031B00083620C0CD0231B0623438362D378002B3D
:1031C00003D15378013B012B02D930BD8161F8E76F
:1031D0008160FAE7FFFFFBFF10B50A00C109002379
:1031E000002904D14309DB0105498C4663441F24AF
:1031F0002040012181401800024B984710BDC04675
:1032000000440041313100007047000010B5054B0B
:103210009847054B9847054B9847054B9847054BF2
:10322000984710BDF52D00000D2C0000093200005C
:103230006505000009320000FEE70000F8B52A4AE3
:103240002A4B9A4211D01A00294B9A420DD2294A90
:1032500003339B1A9B0801339B0000222348224919
:103260008C58845004329A42FAD1234A234B9A4212
:103270000AD2D34321495B1803218B4304339B18A3
:10328000002102C29342FCD11D4AFF211D4B8B43FA
:103290009360FD3990235B001B4AD1501B4AD378C1
:1032A0000325AB4302242343D370D3780C27BB43BD
:1032B00008263343D370164B987B3022904320224C
:1032C00010439873997BB943314399739A7BAA430E
:1032D00022439A730F4A536880210B4353600E4B6D
:1032E00098470E4B9847FEE7F89100000000002039
:1032F0002C020020040000202C0200207804002072
:1033000000ED00E0000000000070004100500041AE
:1033100000480041004000415D330000E10F000023
:103320000300064A1268002A04D0044A1068C31831
:10333000136070470249014A1160F6E7D402002089
:103340007824002001204042704780239B014B607D
:1033500000207047012070470020704770B500269C
:103360000C4D0D4C641BA410A64209D1002605F09B
:103370002FFF0A4D0A4C641BA410A64205D170BD54
:10338000B300EB5898470136EEE7B300EB58984787
:103390000136F2E7DC910000DC910000DC910000D6
:1033A000E0910000002310B59A4200D110BDCC5C22
:1033B000C4540133F8E703008218934200D17047E8
:1033C00019700133F9E7F0B58BB014001D1E129986
:1033D00053DA802424061B191D0014002D230B70C2
:1033E0002023149E03229E43462E07D03300453BE4
:1033F00059424B411099013ACB18109309AB0493F1
:1034000008AB0393139B00920293109B220001933D
:103410002B0000F0EFFE0700472E02D1119BDB07C7
:1034200024D5109BFB180793462E14D13B78302BE4
:103430000CD1002200232000290002F071FE002898
:1034400004D10123109A9B1A139A1360139B079AB5
:103450001B68D3180793002200232000290002F0E4
:103460005FFE302200280DD0079B09933800099B8E
:10347000159ADB1B13600BB0F0BD0023AFE7591C9E
:1034800009911A70099B07999942F8D8EEE7F0B5AF
:103490002B2385B007000C000270861C002901DA7E
:1034A0002D234C427B70092C23DD02ABDD1D6B1EEE
:1034B00020000A21019302F01DFE6B1E30311970AD
:1034C00020000A2102F030FD040009280ADC023D38
:1034D00030342C7002AB07333000AB4204D8C01B31
:1034E00005B0F0BD019DE2E72B7801353370013660
:1034F000F0E73023E4183370B01C7470EFE700007D
:10350000F0B595B00C000A920B931A9D099001F04A
:10351000E7FD036818000D9300F014FD00231293DB
:1035200023680E900C930C99277E2B680722C905FF
:1035300047D59B1893431A0008322A601A685B68C3
:10354000A264E3640122E56CA66C6B005B080F9338
:103550005242A74B30000F9904F0F6FE002800D02D
:1035600006E20122A24B524230000F9902F0E8FD20
:10357000002800D0FCE1002200233000290002F0E6
:10358000D5FD002803D023002D2243331A70994D16
:10359000472F00D8984D032300260C9A236101334E
:1035A0009A4322600B9B13AA009321000A9B09985F
:1035B00000F0F2F9431C00D09CE00120404215B01D
:1035C000F0BD0733B6E780236268DB00511C45D1AC
:1035D000073262600C9A0021134312AA059211AAC5
:1035E0000392232223600691019308A9636852186D
:1035F0000292009332002B0004970998FFF7E3FE34
:1036000020233A0005009A43472A07D1119BDA1C70
:1036100002DB626893425BDD023FFFB21199652FC6
:103620003BD8200001393A0050301191FFF72FFFAD
:10363000129A060083182361012A02DC2268D2074D
:1036400001D501332361232308AA9B181B78002B83
:10365000A8D023002D2243331A70A3E7672F01D08F
:10366000472FB7D1002A16D00C9908A80B43002188
:10367000069112A9059111A903912321091823602C
:10368000019300922B000497029132000998FFF7F2
:103690009AFE0500BAE701229BE7662F19D16368FD
:1036A00000290CDD2161002B02D12268D20702D54E
:1036B00001335B182361119B0026A365C3E7002B30
:1036C00003D101222168114200D09A1C2261F2E745
:1036D0006727119B1298834205DB22682361D2077A
:1036E000E9D50133E6E70122002B01DC9218D21A5A
:1036F0001218EBE72268530508D423692A000A99B7
:1037000009980B9DA847431C29D156E7652F00D87F
:10371000DCE0A06CE16C0022002302F001FD002837
:1037200035D00123354A0A9909980B9DA847431CB7
:1037300000D142E7119B129A934202DB2368DB0718
:103740000DD50B9D0E9B0D9A0A990998A847002547
:10375000431C00D131E7129B013B9D420BDB2368E8
:1037600000259B0700D5FDE0139BE068984200DB35
:1037700025E7180023E7220001231A320A99099845
:103780000B9EB047431C00D117E70135E3E7119BBF
:10379000002B35DC0123194A0A9909980B9EB04782
:1037A000431C00D109E7119B002B05D1129B002B74
:1037B00002D12368DB07D2D50B9E0E9B0D9A0A9986
:1037C0000998B0470026431C00D1F6E6119B5B42E6
:1037D0009E4201DB129B91E7220001231A320A99D3
:1037E00009980B9FB847431C00D1E6E60136EDE788
:1037F000FFFFEF7F588E0000548E0000648E0000A3
:10380000A36D129E9E4200DD1E00002E35DC0023BB
:103810000C93F343DB170F930F9BA76D0C9A334068
:10382000FB1A9A4232DB119B129A93423CDB2368CB
:10383000DB0739D4129E119AF31BB61A9E4200DDA3
:103840001E00002E39DCF7430025FB170C93119A5C
:10385000129B0C999B1A32000A409B1A9D4200DB76
:103860007DE7220001231A320A9909980B9FB84775
:10387000431C00D1A1E60135E9E733002A000A998B
:1038800009980B9FB847431CC1D196E6220001233B
:103890001A320A9909980B9FB847431C00D18CE64D
:1038A0000C9B01330C93B7E70E9B0D9A0A9909986C
:1038B0000B9EB047431CBDD17FE6EA1933000A993D
:1038C00009980B9DA847431CBDD176E6129B012B9E
:1038D00002DC01231A4238D001232A000A990998F0
:1038E0000B9FB847431C00D167E60E9B0D9A0A99BF
:1038F00009980B9FB847431C00D15EE6A06CE16CB1
:103900000022002302F00CFC002808D00025129BA6
:10391000013B9D420DDB220033005032EFE6129B4B
:103920006A1C013B0A9909980B9DA847431CF2D1D8
:1039300043E6220001231A320A9909980B9FB847DF
:10394000431C00D139E60135E1E72A00EAE722000D
:10395000012319320A9909980B9EB047431C00D1E4
:103960002BE60135E368139A9B1A9D42EFDBFBE6D9
:1039700032002B003000290004F0E6FC002800D1C2
:1039800021E6034D472F00D905E6024D03E6C04668
:10399000608E00005C8E0000F7B5150001938A6808
:1039A0000B6900900C00934200DA130022002B6098
:1039B00043321278002A01D001332B6023689B0622
:1039C00002D52B6802332B60062723681F4027D0BF
:1039D000230043331B785A1E93412268920630D449
:1039E0002200019943320098089EB047431C25D01D
:1039F000062320682A68E16803400025042B03D1D0
:103A00008D1AEB43DB171D40A3682269934201DD49
:103A10009B1AED180027BD4220D1002010E001378D
:103A2000E3682A689B1A9F42D2DA220001231932E6
:103A300001990098089EB047431CF0D101204042F4
:103A4000FEBD3020E1184331087021005A1C453179
:103A50000978A218433202331170C1E72200012312
:103A60001A3201990098089EB047431CE6D00137EE
:103A7000D1E70000F0B58BB006920A0043320793FD
:103A8000059004920A7E0C00109B6E2A00D18FE0F4
:103A900017D8632A2CD008D8002A00D199E0582AD8
:103AA00054D026004236327029E0642A01D0692AB7
:103AB000F7D121681A68080623D5111D1960156809
:103AC00025E0732A00D188E008D86F2A29D0702A0F
:103AD000E7D1202209680A43226003E0752A20D03A
:103AE000782ADED122007821453211706C4A30E00C
:103AF0000E001A684236111D1960136833700123D5
:103B000079E04906D9D5111D19600023D55E002D35
:103B100003DA2D23049A6D421370624B0A27039334
:103B20002FE020681968050603D5081D18600D6888
:103B300005E04006F9D50D68081D1860ADB2594B77
:103B4000082703936F2A18D00A2716E045310A7018
:103B5000544A03921A682168101D186015680806F7
:103B600022D5CB0702D52023194321601027002D31
:103B700003D1202322689A4322602300002243338A
:103B80001A706368A360002B5CDB042221689143F8
:103B90002160002D58D1049E002B64D02600039B89
:103BA00042361B7833705EE04806DAD5ADB2D8E70E
:103BB00009681A68080605D5111D1960136862693D
:103BC0001A6006E04906F7D5111D19601368A28A2C
:103BD0001A800023049E236154E01A68111D1960A5
:103BE000166800216268300001F0FCFA002801D05C
:103BF000801B6060636823610023049A137041E0B6
:103C00002369320006990598079DA847431C43D0B5
:103C1000236800259B070FD4099BE06898423DDA92
:103C200018003BE022000123193206990598079EEF
:103C3000B047431C30D00135E368099A9B1A9D4276
:103C4000F0DBE9E7002DA9D0049E2800390002F03E
:103C500067F9039B013E5B5C28003370390002F07A
:103C6000D9F8051EF1D1082F09D12368DB0706D545
:103C700063682269934202DC3023013E3370049B67
:103C80009B1B2361079B09AA00932100069B0598B3
:103C9000FFF782FE431CB3D1012040420BB0F0BDC0
:103CA000778E0000668E00000FB40B4B13B51C68B6
:103CB000002C05D0A369002B02D1200001F07AF975
:103CC00005AB049AA1682000019301F057FE16BCD1
:103CD00008BC04B01847C0465C000020084B70B513
:103CE0001C680500002C05D0A369002B02D1200020
:103CF00001F060F92900A268200001F05BFF70BDAF
:103D00005C00002070B505000E00002804D0836917
:103D1000002B01D101F04EF9AB69AC68002B02D148
:103D2000280001F047F9244B9C420FD16C68A3890D
:103D30001B0702D52369002B20D12100280000F0A9
:103D40005FF900281AD00120404270BD1B4B9C42F5
:103D500001D1AC68EBE71A4B9C42E8D1EC68E6E78E
:103D6000013B0136A360002B04DAA269934216DB03
:103D70000A2914D023685A1C226019703178A3686C
:103D80000029EDD1013BA360002B0FDA22000A319C
:103D9000280000F0DFF8431CD5D00A20D5E7220028
:103DA000280000F0D7F8431CE8D1CCE70A202368AC
:103DB0005A1C22601870C8E7B88E0000D88E000028
:103DC000988E000010B5034B01001868FFF79AFFAA
:103DD00010BDC0465C0000204A424A41802310B515
:103DE0005200DB0000F002F810BD0000F0B51D002D
:103DF0004F4B85B01E6804000F000092002E05D0C6
:103E0000B369002B02D1300001F0D4F8494B9C4239
:103E100050D17468009B022B05D0012B00D984E09F
:103E2000002D00DA81E02100300001F055F8616BCF
:103E3000002908D023004433994202D0300001F019
:103E4000CDFC002363630023A3616360A3891B0689
:103E500003D52169300001F0C1FCA389364A134023
:103E6000A381009B022B5AD003AB02AA2100300091
:103E700001F042F9A3891843A081002D24D1029DAD
:103E8000280001F0A5F90195071E42D1029B01937C
:103E9000AB4239D1012040420223A2891343A381BE
:103EA0000023A36023004733236023610123636160
:103EB00005B0F0BD214B9C4201D1B468AAE7204B6C
:103EC0009C42A7D1F468A5E7002FD9D0B369002B95
:103ED00002D1300001F06EF8009B012B03D1A389C1
:103EE000009A1A43A2810820A3892760276165618F
:103EF000184018D0012018400023984211D06D427C
:103F0000A360A5611800D3E7019801F061F9071ECD
:103F1000C0D08023A289019D1343A381D6E700204E
:103F2000BAE7A560C4E7A060C2E701204042BFE74E
:103F30005C000020B88E00005CF3FFFFD88E00000C
:103F4000988E00000023C25C0133002AFBD1581E6A
:103F500070470000F8B505000E001400002804D0DA
:103F60008369002B01D101F025F8224B9C422DD111
:103F70006C68A369A360A3891B0731D52369002B53
:103F80002ED023682269F7B2981A6369F6B2984274
:103F900005DB2100280000F09FFF002826D1A36840
:103FA0000130013BA36023685A1C22601F706369C3
:103FB000984204D0A389DB071AD50A2E18D1210014
:103FC000280000F089FF002812D00FE00A4B9C4225
:103FD00001D1AC68CDE7094B9C42CAD1EC68C8E777
:103FE0002100280000F00CF80028CAD001267642F3
:103FF0003000F8BDB88E0000D88E0000988E00000A
:10400000364B70B51D6806000C00002D05D0AB695D
:10401000002B02D1280000F0CDFF314B9C420FD184
:104020006C680C23E25E93B219072DD4D90611D423
:1040300009230120336037331343A381404270BD0D
:10404000284B9C4201D1AC68EBE7274B9C42E8D15E
:10405000EC68E6E75B0713D5616B002908D0230005
:104060004433994202D0300001F0B8FB002363636F
:104070002422A3899343A3810023636023692360DF
:104080000823A2891343A3812369002B0BD1A0210C
:104090008022A389890092000B40934203D0210023
:1040A000300001F051F80123A289134011D0002300
:1040B000A36063695B42A361002023698342BED190
:1040C0000C23E25E1306BAD540231343A3810138C3
:1040D000B5E7920700D46369A360EDE75C000020B8
:1040E000B88E0000D88E0000988E0000F0B50369ED
:1040F0000C6989B00700059100269C426DDC0B001D
:10410000013C1433A50003935B190493030014339B
:1041100002935D19049B28681B68591C019301F0E8
:1041200079FE0190B0422DD0039B02989C460696E2
:10413000624608CA9446019A99B251431B0C5343F4
:1041400089190A0C9B18079302881E0C069B89B2DA
:10415000D2180368521A190C6B469B8BCB1A111498
:104160005B18191492B21B041A43049B069104C0F5
:104170006345DDD22B68002B04D1029B043DAB428A
:104180002ED33C610599380001F049FA002823DB61
:104190000025019B029801330399019308C9028805
:1041A00055199AB2AA1A05681B0C2D0CEB1A151496
:1041B0005B191D1492B21B04134308C0049B8B426D
:1041C000ECD2029AA300D3181A68002A04D1029AEA
:1041D000043B9A4209D33C61019E300009B0F0BD16
:1041E0002B68002BCDD1013CC7E71A68002AF2D119
:1041F000013CECE7F0B516001F00446A9DB0049046
:10420000259D06960797002C08D1102000F0E0FFAE
:10421000049B5862446084600460C460049B5B6AD1
:10422000196800290BD05A68012393404A608B60BB
:10423000049801F01AF80022049B5B6A1A60079B3D
:10424000002B1FDA01232B607B005B080793079C80
:10425000B74B220019931A409A4216D1B54B249AB3
:104260001360069B002B03D1240301D100F091FDC4
:10427000B14B269A0A93B14B002A01D000F08FFD72
:1042800000F08FFD00232B60E1E7069E079F0022D0
:1042900000233000390001F043FF051E0ED001233A
:1042A000249A1360A64B269A0A93002A01D100F0A3
:1042B00078FDA44A26990A6000F073FD1AAB0193B9
:1042C0001BAB009332003B00049801F025FA630019
:1042D00005905B0D00D17FE03A039B4C120B144319
:1042E00021009A4A300018959E180022984B03F03E
:1042F00015FD984A984B03F091FA984A984B02F0B2
:1043000049FB040030000D0004F072F8954A964B0A
:1043100003F084FA02000B002000290002F03AFBAF
:1043200004000D0004F030F8002203900023200068
:10433000290001F0FBFE00280ED0039804F058F885
:104340000B0002002900200001F0EAFE03005842A1
:104350005841039B1B1A039301231693039B162BAF
:104360000FD88249DB00C91808684968069A079B7C
:1043700001F0F0FE00284BD0039B013B0393002388
:1043800016931A9B9E1B00230B933300013B0C9347
:1043900004D501239B1B0B9300230C93039B002B41
:1043A00038DB039A0C9B944663440C9300230F92D2
:1043B0000893229B0125092B00D991E0052B02DDF2
:1043C0000025043B2293229B981E032800D991E0EC
:1043D00001F016FD828429761A9B1B9A9E18644B65
:1043E000F218202A0FDD634B0698F318D8404023BB
:1043F0009B1A9C40204304F03DF801235E4C013E93
:104400000919189371E7202306989B1A9840F2E740
:104410001690B6E70B9B039A9B1A0B935342089393
:1044200000230F93C5E701230E93239B002B65DD2B
:104430001F000D93049A546A002262600432110036
:10444000143199425FD96168049800F0D6FE049B4C
:1044500020605B6A1B680A930E2F00D905E1002DCE
:1044600000D102E1069B079C14931594039B002B3B
:1044700000DC85E01A000F213C4B0A40D2009B185B
:104480005C681B6810931194039B02241D11EB06BA
:104490000AD53A4B0D401A6A5B6A1498159902F0D6
:1044A00089FD069007910134344E002D30D1109AC9
:1044B000119B0698079902F07DFD069007917AE01E
:1044C0000123239A0E939446039B63445F1C0D9330
:1044D0003B1EAFDC0123ADE70023A5E70023F0E797
:1044E00000230E952293013B00220D931F001333EE
:1044F00023929FE701230E93023BF5E701230D93DF
:104500001F001A00F4E7616852000131616096E70C
:1045100001231D4208D010981199E418326873687D
:1045200003F07CF9109011916D100836BDE7C0467C
:104530000000F07F0F270000918E0000948E000095
:10454000648E0000658E00000000F03F01FCFFFF5C
:104550000000F83F61436F63A787D23FB3C8608B09
:10456000288AC63FFB799F501344D33F208F000019
:104570003204000012040000000010FEF88E00005B
:10458000039B0224002B16D0149815995D420F232B
:10459000CA4A2B40DB00D3181A685B6803F03EF967
:1045A000002306900791C64E2D11002D00D08CE0FF
:1045B000002B00D081E7169B002B00D191E0069ADA
:1045C000079B10921193109811990022BD4B01F096
:1045D000ADFD002800D184E0002F00D181E00D9BCB
:1045E000002B3EDD10981199039B00225E1EB64BF6
:1045F00003F014F9069007910D9D0134200003F09B
:10460000F7FE069A079B03F009F90022AF4B02F070
:10461000C1F912901391129B139CAD4A10931194FF
:10462000139B9C181194002D5ED1069807990022C7
:10463000A84B03F073FB109A23000690079101F03A
:1046400089FD002800D001E3A34813998446614402
:104650000B0006980799109A01F068FD002800D019
:10466000E8E2149B159C069307941B9B002B00DA31
:1046700057E1039A0E2A00DD53E1904BD2009B18BC
:104680005C681B6808930994239B002B00DBCEE039
:10469000002F00DDCBE000D0CFE20898099900227E
:1046A0008C4B03F0BBF8069A079B01F05DFD3E00C2
:1046B0000897002800D0A4E20A9B0A9A5D1C3123C7
:1046C0001370039B013303939FE20122154205D02F
:1046D000A4183268736803F0A1F801236D1008363E
:1046E00063E7039E3D0089E70A9A691E52191792F3
:1046F0000E9A724BC900002A4AD05B181A685B6890
:104700000020764902F056FC109A119B03F006FB3C
:104710000A9B1090119112930698079903F034FEAA
:10472000040003F065FE02000B000698079903F0F1
:10473000F5FA129B30345D1C1C70109A119B069088
:10474000079101F0F3FC002865D1069A079B002031
:104750005C4903F0E3FA109A119B01F0E7FC002892
:1047600000D0BEE0179B9D4200D17AE710981199C6
:104770000022554B03F052F8002210901191069838
:104780000799514B03F04AF8129506900791C3E739
:10479000591808684968109A119B03F03FF8109067
:1047A00011910A9C179D0698079903F0EDFD129050
:1047B00003F01EFE02000B000698079903F0AEFA04
:1047C000129B0690079130332370179B013400220F
:1047D000A34224D1414B1098119902F0DBF802005A
:1047E0000B000698079901F0B5FC002800D078E08E
:1047F000109A119B0020394903F090FA02000B0037
:104800000698079901F092FC002800D129E76B1E59
:104810001A78302A01D003963FE01D00F7E706988A
:104820000799294B02F0FAFF06900791BBE70A9E11
:10483000089A099B0698079902F0BCFB03F0A4FDB7
:10484000040003F0D5FD089A099B02F0E7FF0B0076
:1048500002000698079903F061FA230030333370A1
:104860000A9B751CEB1A9F424CD102000B0002F010
:1048700091F806000F0002000B000898099901F05A
:1048800055FC00282CD10898099932003B0001F012
:1048900047FC002801D0E30722D40599049800F0D2
:1048A000E4FC00232B70039B249A01331360269BA6
:1048B000002B00D175E21D6073E2C046208F00001E
:1048C000F88E00000000F03F0000244000001C4073
:1048D0000000C0FC000014400000C07C0000E03F6D
:1048E000039E6B1E1A78392A06D10A9A9A4207D17A
:1048F00030231370130001361A7801321A708AE7D8
:104900001D00EEE70022CF4B02F088FF00220023BB
:10491000069007912E0001F003FC002800D187E7E4
:10492000BBE70E9A002A00D187E0229A012A6EDCAA
:10493000189A002A67D0C44A9B18089D0B9C0B9AB2
:104940000121D2180B920C9A0498D3180C9300F002
:104950002AFD0600002C0EDD0C9B002B0BDD0C9AB3
:104960002300944200DD13000B9AE41AD21A0B9232
:104970000C9AD31A0C93089B002B1ED00E9B002B75
:104980005FD0002D11DD31002A00049800F0A4FD55
:10499000059A01000600049800F00EFD059910909C
:1049A000049800F062FC109B0593089B5A1B04D0EE
:1049B0000599049800F090FD05900121049800F0FD
:1049C000F2FC0F9B0890002B3DDD1A0001000498BB
:1049D00000F082FD229B08900025012B3BDC002586
:1049E000069BAB4233D1079B1B03AB422FD1199BD4
:1049F000079A13422BD00B9B013501330B930C9B71
:104A000001330C9323E036231A9A9B1A95E7089BEF
:104A10007D1EAB4206DB5D1B002F0BDA0B9BDC1B04
:104A200000238CE7089B0895EA1A0F9B00259B182A
:104A30000F93F1E70B9C3B0081E7089D0B9C0E9EBA
:104A400088E7089AB4E7229B0025012BC7DD0F9B5E
:104A50000120002B0BD0089B089A1B690F9303338E
:104A60009B00D318586800F055FC2023181A0C9BA3
:104A7000C0181F23184000D1ABE001331B1A042BD0
:104A800000DC9BE01C23181A0B9B24181B180B93AB
:104A90000C9B1B180C930B9B002B05DD1A00059932
:104AA000049800F06BFD05900C9B002B05DD1A00AF
:104AB0000899049800F062FD0890169B002B00D125
:104AC00089E00899059800F0AAFD002800DB82E043
:104AD000039B0A22013B039305990023049800F0ED
:104AE000DDFB0E9B0590002B00D15DE10023310022
:104AF0000A22049800F0D2FB0D9B0600002B02DC7A
:104B0000229B022B6DDC002C05DD31002200049875
:104B100000F034FD06003000002D11D071680498BB
:104B200000F06BFB3100040033690C319A1C9200D9
:104B30000C30FEF737FC01222100049800F01EFD26
:104B40000D9F0A9B013F0B93DB19370006000F9363
:104B500008990598FFF7CAFA39000D9004000598E6
:104B600000F05DFD32000E900899049800F070FD91
:104B700001230C93C36830340500002B04D10100DD
:104B8000059800F04CFD0C902900049800F06DFB96
:104B90000C9B229A134300D089E0069A01331342FA
:104BA00000D084E0392C00D1A3E00E9B002B01DD66
:104BB0000D9C31340B9B5D1C1C7027E0042B00D135
:104BC00069E70B9A1C33D2180B920C9AE418D3188D
:104BD00060E70300F5E7002F3CDC229B022B39DD68
:104BE0000D970D9B002B0CD108990522049800F01D
:104BF00055FB08900100059800F011FD002800DD2C
:104C00005AE5239B0A9DDB430393002708990498E8
:104C100000F02BFB002E00D13FE6002F05D0B7425D
:104C200003D03900049800F020FB3100049800F014
:104C30001CFB32E608952E00E3E7002308931E00D4
:104C4000DFE7C046000024403304000003960895C7
:104C50002E0031E50E9B0D97002B00D053E70A9DE7
:104C600008990598FFF742FA0A9B30300D9A287090
:104C700001350400EB1A9A4278DC151E00DC012590
:104C800000270A9B5D1905990122049800F076FC23
:104C90000899059000F0C3FC00282FDC01D1E30740
:104CA0002CD46B1E1A78302AB0D11D00F9E70E9B68
:104CB000002B07DB1D00229B1D4326D10123069AF2
:104CC000134222D10C9B002B00DC73E705990122D3
:104CD000049800F053FC0899059000F0A0FC00280F
:104CE00004DC00D066E7E30700D463E7392C00D08A
:104CF0005EE70B9B0B9A5D1C392313706B1E1A78B1
:104D0000392A3BD001321A7080E70B9B01330D9397
:104D10000C9B002B05DD392CEBD00D9D01340B9B3A
:104D20004AE70B9B0F9A0D9D1C709342ABD000235A
:104D30000A220599049800F0B1FA002305900A228E
:104D400039000498B74206D100F0A8FA070006001F
:104D50000D9B0B93FCE600F0A1FA31000700002345
:104D60000A22049800F09AFA0600F1E700230A22CA
:104D70000599049800F092FA059071E70A9A9A4210
:104D800005D1039B01330393312313703EE71D00CC
:104D9000B4E70A4B269A0A93094B002A01D0269AB7
:104DA00013600A981DB0F0BD0D9B002B00DD56E787
:104DB000229B022B00DC52E713E7C046888E0000DE
:104DC000908E0000F7B58A8905000C00130760D4A7
:104DD0004B68002B04DC0B6C002B01DC0020FEBDBB
:104DE000E76A002FFAD000232E682B6080235B0136
:104DF0001A4034D0606DA3895B0706D56368C01A7A
:104E0000636B002B01D0236CC01A0200216A0023BF
:104E10002800E76AB847A189431C06D12B681D2BDF
:104E200031D82C4ADA40D3072DD50023636023699B
:104E30002360CB0405D5431C02D12B68002B00D185
:104E40006065616B2E600029C8D02300443399420D
:104E500002D0280000F0C2FC00206063BFE70123FD
:104E6000216A2800B847431CC5D12B68002BC2D04B
:104E70001D2B01D0162B01D12E60AFE74023A28954
:104E80001343A381ABE740230B430120A38140429E
:104E9000A5E70F69002FA1D00B680F60DB1B019302
:104EA0000023920700D14B69A360019B002B00DC1B
:104EB00094E7019B3A00216A2800A66AB0470028BF
:104EC00003DC4023A2891343DFE7019B3F181B1A31
:104ED0000193EAE7010040200B6970B505000C0062
:104EE000002B01D1002070BD002804D08369002B65
:104EF00001D100F05FF80B4B9C4209D16C680C2289
:104F0000A35E002BEED021002800FFF75BFFEAE74D
:104F1000054B9C4201D1AC68F1E7044B9C42EED1B9
:104F2000EC68ECE7B88E0000D88E0000988E000088
:104F300010B5024900F0B2F810BDC046D94E0000CD
:104F4000002310B5040003604360836081814366E1
:104F5000C281036143618361190008225C30FEF75E
:104F60002AFA054B24626362044BA362044BE3629A
:104F7000044B236310BDC046455C00006D5C00001F
:104F8000A55C0000D15C000070B568254A1E554341
:104F90000E002900743100F06BFC041E08D00021C3
:104FA0002A00016046600C30A0606832FEF703FA08
:104FB000200070BD836913B50400002B28D18364E1
:104FC000C3640365134B144A1B68826201939842C1
:104FD00001D101238361200000F020F860602000EF
:104FE00000F01CF8A060200000F018F80022E0603B
:104FF00004216068FFF7A4FF01220921A068FFF7E0
:105000009FFF02221221E068FFF79AFF0123A361AC
:1050100013BDC046508E0000314F0000F8B51E4B46
:1050200007001E68B369002B02D13000FFF7C2FFF2
:105030004836B4687368013B04D53368002B07D049
:105040003668F6E70C22A55E002D0DD06834F2E735
:1050500004213800FFF798FF30600028F0D10C23BE
:1050600004003B602000F8BD012320005B42E38187
:105070000233A38165662560A56065602561656171
:10508000A561082229005C30FEF795F96563A563E8
:10509000A564E564E6E7C046508E0000F7B504005D
:1050A0000700002601914834002C01D13000FEBDDC
:1050B0006368A5680093009B013B009301D52468B9
:1050C000F2E7AB89012B08D90E22AB5E013304D085
:1050D00029003800019B984706436835EBE700003C
:1050E000034B1B68186A002800D10248F030704753
:1050F0005C000020C000002070B50E001D000E23D3
:10510000C95E90B01400002907DA00232B60B38930
:105110001B0611D48023DB000FE001AA00F004FE7F
:105120000028F2DBF022029B12021340054A9B1872
:105130005A4253412B60EDE740230020236010B01A
:1051400070BDC04600E0FFFFF7B502268B89050061
:105150000C00334206D02300473323602361012330
:105160006361F7BD01AB6A46FFF7C6FF0099070010
:10517000280000F07DFB002808D10C22A35E9A05D0
:10518000EFD4032293431E43A681E4E70F4BAB62A7
:105190008023A28920601343A381009B2061636167
:1051A000019B002B0DD00E23E15E280000F0CEFD08
:1051B000002806D00322A38993431A000123134336
:1051C000A381A0893843A081CBE7C046314F0000BE
:1051D00010B5034B0100186800F04AFB10BDC04633
:1051E0005C000020C9B28218904201D100207047B3
:1051F00003788B42FBD00130F6E770B5466A0400B5
:105200000D00002E07D11020FFF7E2FF606246601C
:1052100086600660C660666AF368002B13D0636A16
:10522000AA00DB689B181868002818D101210E001D
:10523000AE40721D9200200000F0C2FA00280CD08F
:10524000456086600DE021220421200000F0B8FABC
:10525000636AF060DB68002BE1D1002070BD02685A
:105260001A6000230361C360F8E770B5446A060062
:105270000D00002C07D11020FFF7AAFF70624460D8
:1052800084600460C460002D07D0736A6A68DB68BC
:1052900092009B181A682A601D6070BDF7B51E0049
:1052A00014239C4607000C0000200D698C446346C3
:1052B00019881B6851431B0C534389190E0C9B1909
:1052C00089B21E0C1B045B186146013008C18C4674
:1052D0008542ECDC002E1BD0A3689D4212DB636884
:1052E0003800591CFFF789FF2100236901909A1C9F
:1052F00092000C310C30FEF755F821003800FFF712
:10530000B4FF019C2B1D9B00E31801355E602561F5
:105310002000FEBD0300020C0020824201D11B04CC
:1053200010301A0E01D108301B021A0F01D10430BF
:105330001B019A0F01D102309B00002B03DB0130CF
:105340005B0000D4202070470722036810B50100DD
:105350001A400DD001240020234205D1023003421F
:1053600003D0E34020000B6010BD9B080B60FBE7FF
:105370009CB21000002C01D110201B0CDAB2002AC4
:1053800001D108301B0A1A0701D104301B099A0702
:1053900001D102309B08DA07E8D45B0801D0013064
:1053A000E4E72020E0E710B50C000121FFF725FF1E
:1053B00001234461036110BDF0B50B69150012694A
:1053C00089B00C00934201DA2C000D0027692E6988
:1053D000A268BB1961680193934200DD0131FFF7B8
:1053E0000CFF030014330093009ABB1994469B00F2
:1053F0009C4413000022049063451CD32A001434FB
:10540000BF00E3191432B600059393190294069372
:10541000069B9A4211D3019B002B06DD04235B42BD
:105420009C4463461B68002B51D0049B019A1800D2
:105430001A6109B0F0BD04C3DEE71488002C1ED049
:105440000026009D029F01CF079508CD039383B2EC
:10545000634319006B46000C9B896043CB1803998A
:105460009B19090C4118180C09180E0C9BB2090461
:105470000B4307990B60059BBB42E4D82E60136871
:105480001B0C03931ED00026009B029C1B680098F7
:1054900007002188039D9BB2694320C82D0C491940
:1054A0008E1931040B433B6008CC03991B0C4B4312
:1054B0007968360C89B25B1805999B191E0CA142BC
:1054C000E6D80360009B043204330093A0E7019BFD
:1054D000013B01939FE700000323F7B5134005004C
:1054E0000E001400002B08D02249013B9A005258AC
:1054F00000233100FFF7D2FE0600A310019336D03F
:105500006C6A002C07D11020FFF762FE68624460CD
:1055100084600460C4606F6ABC68002C07D11649BF
:105520002800FFF740FF00230400B8600360012259
:10553000019B13420AD0310022002800FFF73CFFF4
:10554000070031002800FFF790FE3E00019B5B1032
:1055500001930CD02068002807D1220021002800E8
:10556000FFF72AFF0023206003600400DFE730001C
:10557000FEBDC046E88F000071020000F0B50D00CE
:1055800017002B69541185B0E3180293013301937E
:105590004968AB680390019A934234DB0398FFF7A4
:1055A0002CFE00230200060019001432A3422DDB5A
:1055B000E343DB171C402B001F21A40014192A69A8
:1055C000143392009A180F4024D00131C91B8C4625
:1055D00000211868B84001436046216002CB0434C2
:1055E000C1409A42F5D82160002902D0029B0233C3
:1055F0000193019B0398013B33612900FFF735FEBE
:10560000300005B0F0BD01315B00C4E798001150D7
:105610000133CBE702CB02C49A42FBD8E9E70A691F
:10562000036930B59B1A0ED19200143014318418DE
:105630008918043C043922680D68AA4205D0AA42A0
:10564000924101231343180030BDA042F1D3FAE781
:10565000F0B50D0085B00700110028001400FFF719
:10566000DEFF061E08D101003800FFF7C6FD01234A
:105670004661036105B0F0BD01230193002804DBFE
:1056800023002C001D000023019361683800FFF700
:10569000B4FD2F000022019B2669C3601434B300BF
:1056A000E31802932B6914379B00FB180393030044
:1056B0009446143320CC04CF0192AAB294446A4693
:1056C000614692882D0C8A1A0199090C691A1514E1
:1056D00049190D1492B209040A431A60039AAC46A0
:1056E0000433BA42E6D802991A008C4205D3043A30
:1056F0001368002B0ED00661BCE704CC91B2614464
:105700000D14120C5219151489B212040A43AC4636
:1057100004C3E8E7013EEAE7F7B51D000121089F51
:105720001400FFF76AFD2B036D0006001B0B6D0DC7
:1057300024D10193002C27D068460094FFF704FE83
:10574000009C00281ED0019B20211A00091A8A40C3
:10575000C340224372610193019CB461631E9C416A
:1057600001343461002D18D0124BED1835232D185B
:105770003D60181A099B18603000FEBD802252035C
:105780001343D6E77461E7E701A8FFF7DDFD0124C5
:10579000019B346173612030E4E7074BC018074B6D
:1057A0003860E3189B00F3185869FFF7B3FD6401F4
:1057B000201ADFE7CDFBFFFFCEFBFFFFFFFFFF3F20
:1057C0004A4370B51100140000F052F8051E03D0D2
:1057D00022000021FDF7EFFD280070BD70B5050027
:1057E000002910D00C1F2368002B00DAE4182800D1
:1057F00000F0E4FA1D4A1368002B05D163601460C1
:10580000280000F0DCFA70BDA34209D921686018B5
:105810008342F3D118685B6841182160EEE71300FA
:105820005A68002A01D0A242F9D919685818A04232
:105830000BD120680918581819608242E0D110680D
:105840005268411819605A60DAE7A04202D90C2365
:105850002B60D5E721686018824203D11068526836
:105860004118216062605C60CAE7C046D80200202F
:10587000032370B5CD1C9D43083506000C2D1ED2A8
:105880000C25A9421DD8300000F098FA254A14686A
:105890002100002919D1244C2368002B03D13000AA
:1058A00000F0BEF920602900300000F0B9F9431C77
:1058B0002CD10C233000336000F081FA03E0002D7E
:1058C000DFDA0C233360002070BD0B685B1B1AD439
:1058D0000B2B03D90B60CC18256003E08C420ED152
:1058E00063681360300000F06AFA200007220B3072
:1058F000231D9043C31AE7D05A42E250E4E74B68B5
:1059000063600C00EEE70C004968C2E70323C41C87
:105910009C43A042E0D0211A300000F081F9431CE2
:10592000DAD1C6E7D8020020DC020020936810B567
:10593000013B9360002B05DA9469A34208DBCBB2EC
:105940000A2B05D01368581C10601970C8B210BD1E
:10595000FEF700FBFBE7F8B506000F001400D518B2
:10596000AC4201D1002007E021783A003000FFF777
:10597000DDFF0134431CF3D1F8BD0000F0B59FB04A
:1059800006000F0014000593002804D08369002B43
:1059900001D1FFF70FFB7F4B9F425CD17768BB893A
:1059A0001B0762D53B69002B5FD0002306AD6B61FE
:1059B00020336B761033AB760294029C2378002B55
:1059C0005DD1029BE31A04930DD0049B029A390027
:1059D0003000FFF7C0FF431C00D1CCE06A69049B94
:1059E000944663446B612378002B00D1C3E001220D
:1059F000002352426A6002A95432521801342B60CB
:105A0000EB60AB601370AB65217805226248FFF74D
:105A1000E9FB631C9C46002835D12968CB0604D5D8
:105A2000532302AA20309B1818700B0704D5532368
:105A30002B2002AA9B18187023782A2B2CD0002028
:105A40000A21099B2278303A092A00D86BE0002805
:105A50002AD0099328E0514B9F4201D1B7689EE7B5
:105A60004F4B9F429BD1F76899E739003000FEF712
:105A7000C7FA002899D0012040421FB0F0BD252B65
:105A80009FD001349AE7444B2968C01A0123834010
:105A90000B432B606446B7E7059B181D1B680590F8
:105AA000002B3ADB0993644623782E2B0BD16378C5
:105AB000621C2A2B3FD1059B02341A1D1B680592DC
:105AC000002B35DB0793217803223648FFF78AFB4A
:105AD000002807D0334B2A68C01A40238340134361
:105AE0002B6001342178631C06222F48029329760B
:105AF000FFF778FB002844D02C4B002B2FD12968CE
:105B0000059B0722C90528D59B18934308330593A5
:105B10006B69039A9B186B614FE75B42EB60022352
:105B20000B432B60BFE74B4301349B18012089E7EF
:105B300001235B42C6E7002314000A201A006B60B1
:105B400021783039092903D9002BBCD00792BAE754
:105B50004243013452180123F2E70733D5E705AB7E
:105B600000933A00124B29003000FDF7C9FC039066
:105B7000039B0133CCD1BB895B0600D57BE70B9837
:105B80007BE705AB00933A00094B29003000FDF795
:105B900071FFECE7B88E0000F48F0000D88E000093
:105BA000988E0000FA8F0000FE8F00000135000083
:105BB0005759000070B506000D001400002804D0ED
:105BC0008369002B01D1FFF7F5F9124B9C4211D1EB
:105BD0007468A368013BA360002B05DAA2699342B5
:105BE00012DBEBB20A2B0FD02368E8B25A1C2260FA
:105BF0001D7070BD084B9C4201D1B468E9E7074BAA
:105C00009C42E6D1F468E4E7220029003000FEF768
:105C1000A1F9EEE7B88E0000D88E0000988E000043
:105C2000002370B5064C050008002360FDF778FBE3
:105C3000431C03D12368002B00D02B6070BDC046ED
:105C40007404002070B50C000E25495F00F0B8F810
:105C5000002803DB636D1B18636570BDA389024ACE
:105C60001340A381F9E7C046FFEFFFFFF8B51F001F
:105C70008B8905000C001600DB0505D50E23C95ED7
:105C80000022022300F074F8A389054A280013407B
:105C9000A38132000E23E15E3B0000F01FF8F8BD47
:105CA000FFEFFFFF70B50C000E25495F00F060F8B4
:105CB000A389421C03D1054A1340A38170BD8022F1
:105CC00052011343A3816065F8E7C046FFEFFFFF71
:105CD00010B50E23C95E00F015F810BD70B50500B3
:105CE000080011000022064C22601A00FAF72AFE72
:105CF000431C03D12368002B00D02B6070BDC0462D
:105D000074040020002370B5064C050008002360D1
:105D1000FDF718FB431C03D12368002B00D02B6038
:105D200070BDC04674040020002370B5064C050009
:105D3000080011002360FDF708FB431C03D1236812
:105D4000002B00D02B6070BD74040020002370B5C0
:105D5000064C050008002360FDF7FCFA431C03D144
:105D60002368002B00D02B6070BDC0467404002057
:105D700070B50500080011000022064C22601A00D0
:105D8000FDF7EAFA431C03D12368002B00D02B60F7
:105D900070BDC0467404002082B0002900D101A962
:105DA000101E06D0002B06D013780B601078431E0F
:105DB000984102B0704702204042FAE770477047AE
:105DC00070B50500080011000022064C22601A0080
:105DD000FAF796FD431C03D12368002B00D02B60FB
:105DE00070BDC046740400200B1E04D0FF2A04D9E5
:105DF0008A2303608B3B180070470A700123FAE77F
:105E000002B4714649084900095C49008E4402BC4D
:105E10007047C046002243088B4274D303098B426B
:105E20005FD3030A8B4244D3030B8B4228D3030C6A
:105E30008B420DD3FF22090212BA030C8B4202D30C
:105E40001212090265D0030B8B4219D300E0090A34
:105E5000C30B8B4201D3CB03C01A5241830B8B423D
:105E600001D38B03C01A5241430B8B4201D34B0326
:105E7000C01A5241030B8B4201D30B03C01A52418B
:105E8000C30A8B4201D3CB02C01A5241830A8B4210
:105E900001D38B02C01A5241430A8B4201D34B02F9
:105EA000C01A5241030A8B4201D30B02C01A52415D
:105EB000CDD2C3098B4201D3CB01C01A5241830911
:105EC0008B4201D38B01C01A524143098B4201D34B
:105ED0004B01C01A524103098B4201D30B01C01A76
:105EE0005241C3088B4201D3CB00C01A52418308F0
:105EF0008B4201D38B00C01A524143088B4201D31D
:105F00004B00C01A5241411A00D20146524110467C
:105F10007047FFE701B5002000F0F0F802BDC04671
:105F20000029F7D076E7704703460B437FD4002261
:105F300043088B4274D303098B425FD3030A8B421D
:105F400044D3030B8B4228D3030C8B420DD3FF2287
:105F5000090212BA030C8B4202D31212090265D055
:105F6000030B8B4219D300E0090AC30B8B4201D308
:105F7000CB03C01A5241830B8B4201D38B03C01A4F
:105F80005241430B8B4201D34B03C01A5241030BC6
:105F90008B4201D30B03C01A5241C30A8B4201D377
:105FA000CB02C01A5241830A8B4201D38B02C01A22
:105FB0005241430A8B4201D34B02C01A5241030A99
:105FC0008B4201D30B02C01A5241CDD2C3098B427E
:105FD00001D3CB01C01A524183098B4201D38B01FB
:105FE000C01A524143098B4201D34B01C01A52419E
:105FF00003098B4201D30B01C01A5241C3088B42E3
:1060000001D3CB00C01A524183088B4201D38B00CD
:10601000C01A524143088B4201D34B00C01A52416F
:10602000411A00D201465241104670475DE0CA0F46
:1060300000D04942031000D34042534000229C4606
:1060400003098B422DD3030A8B4212D3FC22890110
:1060500012BA030A8B420CD3890192118B4208D3E6
:10606000890192118B4204D389013AD0921100E048
:106070008909C3098B4201D3CB01C01A524183095C
:106080008B4201D38B01C01A524143098B4201D389
:106090004B01C01A524103098B4201D30B01C01AB4
:1060A0005241C3088B4201D3CB00C01A524183082E
:1060B0008B4201D38B00C01A5241D9D243088B4284
:1060C00001D34B00C01A5241411A00D20146634627
:1060D00052415B10104601D34042002B00D549428B
:1060E000704763465B1000D3404201B5002000F0CA
:1060F00005F802BD0029F8D016E770477047C04682
:106100008446101C62468C46191C634600E0C0465B
:106110001FB501F021FB002801D40021C8421FBD9A
:1061200010B501F07BFA4042013010BD10B501F00E
:1061300013FB002801DB002010BD012010BDC0466C
:1061400010B501F009FB002801DD002010BD012081
:1061500010BDC04610B501F09BFA002801DC0020FC
:1061600010BD012010BDC04610B501F091FA002805
:1061700001DA002010BD012010BDC046002B11D156
:10618000002A0FD1002900D1002802D00021C943E4
:10619000081C07B4024802A14018029003BDC04683
:1061A0005DFFFFFF03B4684601B5029800F030F8C8
:1061B000019B9E4602B00CBC7047C046F0B5CE466F
:1061C000474615042D0C2E0080B50704140C3F0C17
:1061D0009946030C7E435D43674363437F19340C48
:1061E000E4199C46A54203D980235B029846C44427
:1061F0004B46514343433604360C250C2404654476
:10620000A4195918491920000CBC90469946F0BDB4
:10621000F0B557464E464546DE46E0B5040083B02D
:106220000D00924699468B422FD82CD049465046B5
:1062300002F0C8F929000600200002F0C3F9331A61
:106240009846203B9B4600D574E053465A469340FF
:106250001F005346424693401E00AF4229D826D025
:106260005B46A41BBD41002B00DA79E0002200232D
:106270000092019301235A46934001930123424621
:106280009340009319E08242D0D90022002300926B
:1062900001930C9B002B01D01C605D60009801995C
:1062A00003B03CBC90469946A246AB46F0BDA34223
:1062B000D6D900220023009201934346002BE8D058
:1062C000FB0772081A4346467B080EE0AB4201D139
:1062D000A2420CD8A41A9D41012024196D4100212D
:1062E000013E24184D41002E06D0AB42EED9013EAE
:1062F00024196D41002EF8D15B46009801990019D0
:106300006941002B22DB2B005A46D3402A00444629
:10631000E2401C005B461500002B2CDB26009E4053
:10632000330026004746BE403200801A9941009053
:106330000191AEE7424620239B1A5246DA4041467D
:1063400013004A468A4017001F4382E74246202333
:106350009B1A2A0046469A402300F3401343D5E790
:106360004246202300219B1A002200910192012223
:10637000DA40019282E74246202326009B1ADE4043
:106380002F00B446974066463B003343C9E7C046FA
:10639000F8B557464E464546DE46E0B5470246004C
:1063A00088467F0A360EC40F002E47D0FF2E24D019
:1063B000FB008027FF041F43002399469A467F3E37
:1063C00043465D025800DB0F6D0A000E984643D02D
:1063D000FF283BD0EB0080250022ED041D437F38D1
:1063E0003618731C41469B464B46614013430F2BA6
:1063F00064D875489B00C3589F46002F42D108239C
:106400009946063BFF269A46DAE74146022A28D0FB
:10641000032A00D1CEE0012A00D0ACE011400020D8
:106420000022CCB24002D205400AE40710432043C8
:106430003CBC90469946A246AB46F8BD002F15D10C
:1064400004239946033B00269A46B9E7FF2002221F
:10645000002DC5D00322C3E7002D19D10020012251
:10646000BEE70124FF220C400020DBE7380002F0E9
:106470008BF87626431F9F4000237642361A9946B2
:106480009A469DE70C239946093BFF269A4697E7D3
:10649000280002F079F8431F9D4076235B42181ACA
:1064A00000229DE780200024C003FF22BAE73D00C0
:1064B0005246ABE73D0021005246A7E73B0C9C4605
:1064C0002A04120C2B0C1400604665463F043F0C56
:1064D0007C4342435D437B43270C9B18FF18BA4221
:1064E00003D980235B029C46654424043A04240CAF
:1064F000121993015C1EA3413F0C920E7D191A43A1
:10650000AD0115432B0104D501235E466A081D40E9
:10651000154332007F32002A25DD6B0704D00F239C
:106520002B40042B00D004352B0103D53200274B20
:1065300080321D40FE2A94DC0124A801400AD2B218
:106540000C406FE78020C003074207D0054205D109
:1065500028434002400A4446FF2263E73843400292
:10656000400AFF225EE70124A31A1B2B05DD0C4025
:106570000022002056E75E46CBE72A002020DA40C2
:10658000C31A9D402B005D1EAB4113435A0704D034
:106590000F221A40042A00D004335A0104D50124E2
:1065A00001220C4000203DE701249B01580A0C40C9
:1065B000002237E780200124C00328434002400A1C
:1065C0000C40FF222EE7C04610910000FFFFFFF7AE
:1065D000F0B54F46D64646464400C0B5C20F470206
:1065E0004802400A844666467B0A4800C90F9A461C
:1065F000240E1500DB00000E8946F600FF2800D1AE
:106600008FE001214F464F403900914266D0221A57
:10661000002A00DC9DE000283DD1002E00D18BE057
:10662000511E002900D0B5E001249B1B5A0144D51E
:106630009B019F09380001F0A7FF0538874084427D
:1066400000DD96E0041B3A0020200134E240041BE8
:10665000A7403B005F1EBB41002413435A0704D0F0
:106660000F221A40042A00D004335A0127D50134DE
:10667000FF2C00D179E001229B015B0AE4B22A40A1
:106680005B02E405580AD207204310431CBC904625
:106690009946A246F0BDFF2CE0D08021C9040E43EC
:1066A0001B2A7BDC31002020D140821A9640721ECA
:1066B00096410E439B1B5A01BAD45A07D0D10122EE
:1066C000DF082A40FF2C33D1002F00D1A8E080231F
:1066D000DB033B435B025B0AFF24D1E7211A00295D
:1066E0004CDD00282AD0FF2CB8D08020C0040643FF
:1066F0001B2900DDAFE030002027C840791A8E400A
:10670000711E8E4106439B195901D6D50134FF2CC9
:1067100000D185E001227A491A405B080B401343FF
:106720009CE7002E00D070E76BE73B1EC5D100222E
:106730007B025B0AE4B2A3E714008FE7002E4DD082
:10674000481E002857D19B1901245A01B5D50224AF
:10675000E0E7002A25D1621CD2B2012A72DD9F1B1C
:106760007A0135D5F71A0D0064E7012200232A408B
:1067700086E73B00634A241A13406FE700296CD177
:10678000611CC8B201284EDDFF2949D09B195B0866
:106790000C0063E7FF2A41D00A0081E701269B1B1A
:1067A00089E7002C1CD0FF2821D08024E404524229
:1067B00023431B2A00DD96E01C002025D440AA1AA2
:1067C00093405A1E93412343F31A04000D002DE712
:1067D000002F00D02EE700220024A9E70C003DE79F
:1067E000002B58D0D243002AEED0FF28E1D133004D
:1067F000FF240D0032E7FF2910D0010078E7002BBD
:106800006ED0FF24002E00D128E780225146D2030B
:10681000114203D06146114200D13300FF241DE72D
:10682000FF2400232CE7002CE9D1002B63D0002E9D
:1068300000D113E79B195A0100D43EE7314A0C00FE
:1068400013400BE7002C1ED1002B2FD1002E4FD070
:1068500033000D0002E7012655E7002C1FD1002B65
:1068600043D0C94300290BD0FF2839D01B2944DC71
:106870001C002027CC40791A8B40591E8B412343A2
:106880009B19040040E7002B1AD1002E24D1802749
:106890000022FF031BE7330004000D00DEE6FF28A3
:1068A0001ED08024E40449422343DFE7002E00D1B8
:1068B000D4E69F1B7A0100D437E7F31A0D00CDE62A
:1068C000FF24002E00D1C9E680225046D203104298
:1068D000A4D060461042A1D133000D00FF24BDE6D4
:1068E0003300FF24BAE601236EE733000400B5E667
:1068F000002700221CE73300B0E60123C0E7C046B2
:10690000FFFFFF7DFFFFFFFB10B5041E27D001F046
:106910003BFE9E231B1A962B0ADC9622D21A944029
:106920006402640ADBB26402DB05600A184310BD2E
:10693000992B17DC9922D21A002A27DD94402200D5
:10694000134C1440510704D00F210A40042A00D0F0
:106950000434620112D4A401640ADBB2E3E7002329
:106960000024E0E7B9222100D21A91400A00511E0A
:106970008A410521091ACC401443DBE7044B1C4033
:106980009F23A4011B1A640ADBB2CCE72200D7E7DD
:10699000FFFFFFFBF8B54546DE4657464E460C0363
:1069A000E0B54E00C90F88460D00610A440F0C4344
:1069B000C70019035800DB0F9B464B0A510F0B43CE
:1069C000760D400D1900D200D84500D1AEE0351A41
:1069D000002D00DCF6E000280FD1134300D1DBE0EE
:1069E0006B1E002B00D037E1BA1A9742BF41641AE0
:1069F0007F42E41B0126170024E0C64B9E424DD087
:106A000080231B041943382D00DD07E11F2D00DD15
:106A100038E12020431B9A460B005046834099469C
:106A200013004846EB401843030050468240501E76
:106A30008241E9401A43BA1A611A9742A4411700E9
:106A400064420C1B230262D56402650A002D00D14A
:106A5000DFE0280001F098FD0300083B1F2B00DD5C
:106A6000D2E020223C00D21A9D40D4409F402543D2
:106A70009E4200DDC4E09E1B731C1F2B00DDF1E075
:106A8000202238002900D21AD840914097402C008B
:106A90000143781E8741DC4000260F437B0709D065
:106AA0000F233B40042B05D03B1DBB42BF417F421F
:106AB000E4191F0023022CD5964B01369E4200D1CB
:106AC0009AE04546944BFF081C4060077605640237
:106AD0000743240B760D00212403230B0C0D8F4A52
:106AE00024051C431440330523435B00ED075B087A
:106AF0002B43380019003CBC90469946A246AB4651
:106B0000F8BD6446044300D111E2040067467B07E8
:106B1000C6D145466007FF080743E4087D4B9E4207
:106B200030D024037605240B760DD4E7331A9A4629
:106B3000002B78DD002831D076488642AED0802008
:106B4000000401435346382B00DCE9E00A43511EA0
:106B50008A410021D219BA42BF4109197C4217006B
:106B60000C192302D3D56B4B01369E4200D13AE17A
:106B70000120694B1C407B0807401F43E007074387
:106B800064088BE723003B4300D1CBE18022120352
:106B900014432403240B9EE72E007FE708001043D4
:106BA00000D1B4E0581E002800D0DEE0BA18BA4286
:106BB0009B4164185B42E418170001262302A6D506
:106BC0000226D5E7002D6ED1701C4005400D01282E
:106BD00000DCF9E0B81A844687428041E51A404259
:106BE0002D1A280200D489E0D71BBA4292411C1BFF
:106BF0005242A51AD84629E74546002400276AE7ED
:106C0000454CF61A2C4049E73D00283885400027BE
:106C10002EE7380001F0B8FC20301DE70A43511E72
:106C20008A41002107E7002B00D0F3E0701C4305E8
:106C30005B0D012B00DCADE0364B984200D1D1E07A
:106C4000BA18BA42BF4164187F42E419E7075208F4
:106C500017436408060021E72E48854200D193E0DF
:106C60001D00D0E629001F3EF140202B00D18DE011
:106C70004022D31A9D402F437D1EAF4100240F4375
:106C8000002644E72B000800203BD8400300202DBD
:106C900000D17DE04020451BA9400A43511E8A4196
:106CA00000211A43C7E6002E50D01A4EB04257D0EA
:106CB00080266B429946360434434B46382B00DD20
:106CC000D6E01F2B00DD35E12026F51A2600AE4068
:106CD000B2463E00DE40AC46350056462E43654681
:106CE000AF407D1EAF41DC403743D71BBA429241D3
:106CF0000C1B5242A41A0600D846A3E66446674617
:106D00002C4300D0A2E600250026002706E71E003F
:106D1000C4E6C046FF070000FFFF7FFFFFFF0F80B4
:106D20001F2B63DC2020C31A080098409C46834632
:106D300053461000D84003005846184363469A4013
:106D4000531E9A4153460243D94003E726003E436F
:106D500006D0EB439946002BC7D0944EB042ACD13D
:106D60000C0017000600D84698E6904B9A450BD0C9
:106D70008246E7E6002800D09EE01800104300D1CC
:106D8000E9E01C001700D846884E87E6002572E728
:106D9000002182E723003B43002E00D0ABE0002B14
:106DA00000D1E7E00B00134300D177E6BA18BA42EE
:106DB000BF4164187F42E419230200D4F2E07C4B07
:106DC00017001C40060069E620003843002ED1D190
:106DD00000285BD11C00144300D1A8E01C00170060
:106DE000D8465BE606000024002797E650460B00D5
:106DF0002038C34099465346202B00D195E04023CC
:106E000050461B1A99400A43511E8A414B460021A5
:106E10001A439FE6002E30D126003E4367D0DB4365
:106E20009A46002B1CD0614EB04260D05346382B9E
:106E300000DD96E01F2B00DD9FE02026F31A2600E0
:106E40009E409C46B34653463E00DE4033005E46BD
:106E50001E4363469F407B1E9F415346DC403743A1
:106E6000BF189742924164185242A418060078E66F
:106E700027437C1EA741002437E74C4EB04236D052
:106E800080265B4236049A463443CFE7180010430D
:106E900000D103E6B81A84466745AD41E01A6D4259
:106EA000401B050200D42CE6D71BBA4292411C1BA2
:106EB0005242A41AD846F1E51800104300D163E706
:106EC000F808670707438020E4080003044208D05D
:106ED000DD08054205D1D208590711430F002C00E7
:106EE000D8467B0FE4001C43FF00304ED6E50C0073
:106EF00017000600D2E5002B38D00B00134300D159
:106F000042E7F808670707438020E40800030442CB
:106F1000E7D0CB080342E4D1D208490711430F0060
:106F20001C00DEE700270024D5E500216BE70025E3
:106F30000027F3E54E462500203EF5404B462E0047
:106F4000202B2DD04025ED1AAC4027437C1EA741B5
:106F500000243743C9E6802400252403134E00276C
:106F6000DCE527437C1EA741002479E70C001700CD
:106F70000E4E93E50C00170090E556462300203E88
:106F8000F34099465346202B0ED0402356469B1B78
:106F90009C4027437C1EA7414B4600241F435FE7CC
:106FA0000024D2E71700B2E50024F2E7FF07000053
:106FB000FFFF7FFFF0B557464546DE464E46E0B53B
:106FC0004C000E0387B0834692461D008046360B68
:106FD000640DCF0F002C4FD06F4B9C4235D08023D7
:106FE000420F1B04F600134333439946C3009846EF
:106FF0006A4B00269C460023644403932B031B0B1F
:107000009B466B00ED0F50465B0D01955ED0624ACA
:10701000934253D05A46D1008022400F12040243BB
:107020000A4393465246D1005C4A94460022634488
:107030003800684084460290E41A16430F2E00D9A7
:10704000B4E0574BB6009B599F4603003343994623
:107050006CD100239846023308260393CEE7CB4633
:107060004146039A0197022A65D1019B4A4C9C46EE
:107070000023002298466BE00300334399464ED02C
:10708000002E00D1BCE1300001F07EFA03000B3B82
:107090001C2B00DDACE11D22D31A5A460100DA4058
:1070A00008398E401300334399465B468B4098461F
:1070B00000233C4C0026241A03939FE751465A466E
:1070C000114329D1002293460232B1E759460143C8
:1070D0001ED05B46002B00D19EE1584601F054FAC9
:1070E00003000B3B1C2B00DD8FE102005946083AE0
:1070F00091408B461D21CB1A5146D9400B00594671
:107100000B4351469B469140264B00221B1A8FE7AA
:10711000002301229B468BE75146032288E7002388
:107120009846013304260024039367E70323B146FE
:1071300003930C2662E7032A00D15CE2019B012A3B
:1071400000D0E4E113409C4600230024002298462E
:1071500000211203130B0A0D12051A432305124CCA
:1071600040462240134362465B00D2075B0813434C
:10717000190007B03CBC90469946A246AB46F0BD0C
:10718000002380229C4612039846034CE0E700232C
:10719000014C00229846DBE7FF07000001FCFFFFDF
:1071A000509100000DFCFFFFFFFF0F80D94500D973
:1071B00039E100D134E1002346464D469A46013C70
:1071C0005B460A0E1B021A430B02170C03931304AF
:1071D0001B0C3900280090460193FEF71BFE0200AD
:1071E000019B83465A43280039009146FEF798FEDA
:1071F000350C09040D43A9450DD95B464544013BB7
:10720000A84500D93AE1A94500D837E102235B42FD
:107210009C464544E3444B46EB1A3900180004935E
:10722000FEF7F8FD019B0500434339000498994699
:10723000FEF776FE330409041B0C0B43994509D96C
:1072400043446A1E984500D91AE1994500D817E1D0
:10725000023D43444A469B1A5A4612042A43039964
:107260009346100C0A0C914609045A46090C4E46E6
:107270000D001204120C45430591514372437043B3
:1072800052190E0CB218954203D980256D02AC46F6
:107290006044150C09041204090C28185218834282
:1072A00000D2CEE000D1C8E01D1A53469E1AB24566
:1072B00092415242AB1A9A46984500D117E13900E3
:1072C0001800FEF7A7FD019B050043433900504617
:1072D0000493FEF725FE04980B04310C19438842F1
:1072E00009D941446B1E884500D907E1884200D87E
:1072F00004E1023D4144049BCB1A18003900049379
:10730000FEF788FD019B82464343390004980193B0
:10731000FEF706FE01980B043104090C194388425C
:107320000DD953464144013B884500D9E8E08842E5
:1073300000D8E5E002235B429C464144E244019BC5
:107340002D04CE1A51462943059D4F462A000B04B1
:10735000080C1B0C5A4345437B4378435B19170CBD
:10736000FB189D4203D980256D02AC4660441D0C7C
:1073700012041B04120C28189B18864200D293E0BA
:1073800000D18EE001231943A04BE318002B00DC51
:1073900099E04A0700D09EE05A46D20106D55A46E7
:1073A0009B4B1A4080239346DB00E318994A934293
:1073B00068DD0123029A984C1A40002394469846AF
:1073C0000022C5E680224B46120313420AD05B46D8
:1073D000134206D11A431203120BAC4688468E4C58
:1073E000B6E64B461A431203120BBC468A4CAFE674
:1073F00003005A46283B9A4000239146984657E698
:10740000584601F0C1F8203040E603005246283BC0
:107410009A400021934677E601F0B6F820305FE607
:10742000884500D2C7E64B46DE075D0843465B0849
:107430001E434346DB079A46C2E60025924500D329
:1074400033E7039E5946B446E244B245AD416D422E
:107450004544EB180139984507D2984200D97FE09E
:1074600000D1BCE01D1A8B461FE79845FAD1039D59
:107470005545F2D943468B461D1A16E79B46CAE688
:107480001500E7E65A46C90852070A435B059046CD
:107490005C0D5A460123029952021940120B8C4688
:1074A00056E6002B00D16FE746444A1EB04529D965
:1074B0001100864200D065E7039A934200D061E74D
:1074C00062E7012149420120C21A382A21DD029BCC
:1074D00003409C4638E60F220A40042A00D15BE7AD
:1074E0000A00111D914292415242934454E7474B86
:1074F000E318002BE5DD01225242F2E71D00FAE617
:107500009A461CE7B04239D86ED011003AE7029390
:107510003AE71F2A3CDC20239B1A0C00584699406E
:1075200098404B1E99415B46D440D34020430843CA
:107530001A00430709D00F230340042B05D0010094
:10754000081D88429B415B42D21813023AD50123A1
:10755000029A01241A400023944698460022F7E537
:10756000022149428C46039DE344AC46E244AA45CD
:10757000AD416D424544ED182D1A96E68A1E0399D9
:107580004D008D42894149424144761803958FE769
:107590001F204042C31A5846D8400300202A28D052
:1075A00040205D46821A954029434A1E9141194365
:1075B000072300220B4009D00F2300220B400800B4
:1075C000042BBDD1010053075202120BC908194305
:1075D000012388460299002419408C46B8E552459B
:1075E000BED88B46002560E6039D9D42C6D31100A0
:1075F00062E70025D8E780225B4612031A43019B0D
:107600001203120B9C468846034CA1E5FF030000C1
:10761000FFFFFFFEFE070000FF070000F0B54F462A
:107620004646D6465C00C0B51F03DB0F9A46174B93
:107630000E034D0084468046360B6D0DC90F9146F2
:107640003F0B640D01209D4208D09C4201D0A54211
:107650000BD01CBC90469946A246F0BD634633430E
:10766000F7D1AC42F5D13A43F3D10120BE42F0D17B
:10767000C845EED1514507D0002DEAD163461E43DF
:107680003000461EB041E4E70020E2E7FF070000BB
:10769000F0B54546DE4657464E46E0B51F033D0B66
:1076A0002C4F0E034C00AB465D008446360B640D38
:1076B000C90F90466D0DDB0FBC422AD0254FBD424D
:1076C0002DD0002C0FD130430700814678427841FD
:1076D000C0B2002D17D15F463A4314D14B4600206B
:1076E000002B0AD006E0002D02D15846024301D0FB
:1076F000994218D04842012108433CBC9046994623
:10770000A246AB46F0BD0028F2D00120013B184351
:10771000F3E737000743D1D002204042EDE75F4650
:107720001743CED0F8E7AC42E4DC03DA481E01216F
:107730000843E2E75E45DDD806D000205E45DCD296
:107740000123481E1843D8E7C445D3D80020C445B8
:10775000F6D3D2E7FF070000F0B54E464546DE46B9
:1077600057465C00E0B51F03DB0F99462A4B0E031A
:107770004D00C90F8446360B6D0D8B4690463F0B6E
:10778000640D9D4220D0244B9C4222D0002D12D16A
:10779000304343424341DBB2002C1FD0002B0CD0BE
:1077A0004B460120013B034318003CBC90469946E0
:1077B000A246AB46F0BD002C16D0CB4517D05B4699
:1077C000594201230B43EFE7310002230143EBD180
:1077D000D9E7390002231143E6D1D7E73A43DDD197
:1077E00000230028E0D0EAE73A43E6D1E7E7A542E4
:1077F000E5DC05DBBE42E2D807D00023BE42D3D28F
:107800005946012301390B43CEE7C445D7D800239D
:10781000C445F5D3C8E7C046FF070000F0B557469A
:107820004546DE464E46E0B50C0398464E00230B17
:1078300087B0070092469B46760DCD0F002E6BD089
:107840006D4B9E4235D080245B46420F2404DB0002
:1078500014431C43C3009946684BA3469C4600232F
:1078600000276644029343461C035A00DB0F504630
:10787000240B520D984600D176E05F4B9A426DD0B2
:107880008023410F1B040B435C49E4008C461C43DE
:10789000C300002062444146B6186940721C019141
:1078A000944607430F2F00D9B0E0554ABF00D25984
:1078B00097465B460343994600D087E000239B46EA
:1078C000023308270293CEE742460192022867D08E
:1078D000032800D10EE2012800D062E10023002439
:1078E0000022994601990140CDB2002112030B0DEF
:1078F000120B1B051343434A240513401C43640029
:10790000ED0764082C434846210007B03CBC904674
:107910009946A246AB46F0BD034399464FD05B461D
:10792000002B00D189E1584600F02EFE03000B3BEE
:107930001C2B00DD7AE11D22D31A3A0001005C46BF
:10794000DA4008398C4013008F4023439B46B946E8
:1079500000232D4E0027361A029384E75346234313
:107960002AD10024022096E75346234320D0002C3E
:1079700000D157E1200000F007FE03000B3B1C2B59
:1079800000DD49E11D21CB1A51460200D940534682
:10799000083A944093400C431B4A121A00207AE79D
:1079A0000125019B144C1D400023002299469CE7B1
:1079B0000024002201206EE7534603206BE70023DA
:1079C0009B4601330427002602934CE7032381469C
:1079D0000C27029347E780220023002512039946D3
:1079E000054C82E75C464B4602986FE75C464B4687
:1079F000019502986AE7C046FF07000001FCFFFFFF
:107A000090910000FFFF0F800DFCFFFF4A464946A2
:107A1000170C1A0C1B041B0C08041900000C414322
:107A20001500884619007D4379430395894629004E
:107A3000150045434D44029545462D0CAA46029D2E
:107A40005544A94506D98A46802149028946CA4437
:107A500051460391290C0491414609042D04090C57
:107A600088462900250C24044144240C059121005A
:107A700041438846210079438A4668434146504441
:107A80008146080C48446F43824503D9802149024E
:107A900089464F44010C89463900494402914146C8
:107AA0000F0404993F0C88460004C01980444146E5
:107AB000049159460F0C0904090C884659438A461B
:107AC00039005143894641464A435146090C8B4689
:107AD0007B43D2185A44934203D980235B029B46CE
:107AE000D94451460904090C8A46414661437C4306
:107AF000130C12044B445244A1468A463C004146B2
:107B00006C434D4351464D440F0C7D19A94503D993
:107B10008021490288464444049F0399B846414461
:107B20008B468345804141428846514608042F04D4
:107B3000000C3F185846029910188946904292410D
:107B40004F44BA46524299469346C244D144CB442C
:107B50008F42BF41C245894199459B41934592411E
:107B60007F4249422D0C52420F435B4213437F191F
:107B7000FF185B463C19DB0D059A64021C43430267
:107B800013435D1EAB415A46C00D034352021343DB
:107B9000E20156D501205A0803401343E20713437C
:107BA00064085A48604400284DDD5A0709D00F2266
:107BB0001A40042A05D01A1D9A429B415B42E418E0
:107BC0001300E20104D58020514AC00014406044F3
:107BD000504A904200DDE3E60125DB0862071A43C4
:107BE0006402019B9146220B4405640D1D407CE616
:107BF000802259461203114208D0144206D1224372
:107C00001203120B45469946434C6EE65B461A43F7
:107C10001203120B404C68E603005446283B9C407C
:107C20000023B9E600F0B0FC2030A6E60300283BB4
:107C30009F400023BB4699468AE600F0A5FC203011
:107C400074E6B446ADE701252A1A382A06DD019B01
:107C500000241D4000230022994646E61F2A21DC0D
:107C600020252000AD1A1E00AB40A840D6405D1E66
:107C7000AB4130431843D440430709D00F2303409E
:107C8000042B05D00300181D98429B415B42E41869
:107C9000230221D50125019B01241D400023002240
:107CA000994622E61F2521006D42281AC14008008E
:107CB000202A1DD05F35AA1A944023435C1EA3419D
:107CC000072503431D400022002D09D00F22002468
:107CD0001A401800042AD6D1030065076402220B5B
:107CE000DB082B4301259946019B00241D40FCE540
:107CF0000024E2E7802201251203224301991203A6
:107D0000120B0D409946044CEFE5C046FF030000FE
:107D1000FFFFFFFEFE070000FF070000F0B546462C
:107D2000D6464F460C03C0B5CD0F4E00610A440F36
:107D30000C43C1005800400D84468A460F001903C9
:107D4000500F490A0143C648760DA846DB0FD20002
:107D5000844500D1D8E001204340AB4200D1A6E0E9
:107D60006046351A002D00DC05E1002810D10B001B
:107D7000134300D1D7E06B1E002B00D04BE15346DC
:107D80009F1ABA458041641A4042241A01261EE017
:107D9000B34B9E4248D080231B041943382D00DD8D
:107DA00019E11F2D00DD4CE120230F005B1B1000AB
:107DB0009A409F40E840531E9A41E94007431743C9
:107DC0005346DF1B611ABA45A44164420C1B2302CF
:107DD00000D4C5E06402650A002D00D1F6E0280059
:107DE00000F0D2FB0300083B1F2B00DDE9E020225E
:107DF0003C00D21A9D40D4409F4025439E4200DD66
:107E0000DBE09E1B731C1F2B00DD0AE120223800E3
:107E1000D21A290097402C009140D8407A1E9741F1
:107E2000DC40002601430F437B0709D00F233B4072
:107E3000042B05D03B1DBB42BF417F42E4191F000C
:107E4000230225D5864B01369E4200D1AFE0854BFB
:107E500001251C4043466207FF086402760517436C
:107E6000240B760D1D4000212403230B0C0D7E4AAC
:107E700024051C431440330523435B00ED075B08D6
:107E80002B43380019001CBC90469946A246F0BD11
:107E9000012543466207FF081743E4081D40704B65
:107EA0009E4236D024037605240B760DDBE763462D
:107EB000F31A002B00DC94E06046002835D06848B7
:107EC0008642B1D080273F043943382B00DCFDE0E7
:107ED0000A43170000217A1E9741574457458041B5
:107EE000091944420C1923023AD55D4B01369E42D2
:107EF00000D14BE101225B4B1C407B0817401F4324
:107F0000E207174364088FE70800104300D024E716
:107F100021E723003B4300D1B9E18022120314433F
:107F20002403240B9FE72E007EE70800104300D1B6
:107F3000CAE0581E8446002800D0E7E0524452456B
:107F4000804164184042241817000126230207D5F7
:107F50000226CFE764462C4300D1B3E12C006746EC
:107F60007B0700D062E76307FF081F4301254346F4
:107F7000E4081D4093E7002D78D1751C6D056D0D4B
:107F8000012D00DCF2E05046801A8245BF41651A9F
:107F90007F42ED1B8446280200D48CE05046171A1D
:107FA000BA4292410C1B5542651B984614E70125C5
:107FB000434600241D40002755E72A4CF61A2C4062
:107FC00032E73D0028388540002717E7380000F0E9
:107FD000DBFA203006E70A43170000217A1E97419A
:107FE000EEE6002B00D0E5E0731C9C465B055B0DC4
:107FF000012B00DC9FE01A4B9C4500D1C5E05244A8
:1080000052458041641840422418E707520817433C
:108010006408664608E71248854200D185E01D00E5
:10802000BCE629001F3EF140202B00D17FE040221A
:10803000D31A9D402F437D1EAF4100240F430026DD
:108040008EE72B000F00203BDF40202D71D0402316
:108050005D1BA9400A43511E8A4100211743AFE628
:10806000FF070000FFFF7FFFFFFF0F80002E3ED0C5
:10807000B34EB44545D0802636046D423443382D86
:1080800000DDA8E01F2D00DD1FE12026270050465F
:10809000761BB740E84007435046B040461EB0410B
:1080A000EC403843171ABA4292410C1B5242A41AB0
:1080B000664698468BE6644667462C4300D08BE6BE
:1080C000002500260027EAE61E00ADE61F2B60DC37
:1080D0002027F81A0F00844687401000D840074335
:1080E00060468240501E8241D9401743F5E6260083
:1080F0005046064305D0ED43002DD3D0904EB445F5
:10810000BDD10C001700664698468DE68C48834228
:108110000BD06346D9E6002D00D096E0080010434E
:1081200000D1E2E00C0017009846854E7CE6002561
:1081300080E700218EE7230050460343002E00D045
:10814000A8E0002B00D1DEE00B00134300D16BE66A
:1081500052445245804164184042241817002302BB
:1081600000D4FDE6774B66461C405DE62500504690
:108170000543002ECFD1002D4FD10C00144300D168
:10818000A0E00C00170098464EE666460024002743
:1081900085E61F000800203FF8400700202B00D193
:1081A0008EE04020C31A99400A43511E8A410021A3
:1081B000174392E6002E14D126005046064362D0A3
:1081C000DB43002B5CD187189742924164185242DE
:1081D000A418664687E650462043441EA04100246A
:1081E00060E7574EB4454ED0802636045B42344398
:1081F000382B00DD7FE01F2B00DD8BE020262700E1
:108200005046F61AB740D84007435046B040461E85
:10821000B0410743DC40BF18D6E70D00154300D13D
:1082200002E65046801A8245BF41651A7F42ED1B27
:108230008446280200D48DE65046171ABA4292416D
:108240000C1B5242A41A9846EEE50D00154300D1CE
:108250006BE750466707C00807438020E408000327
:10826000044207D0CD08054204D12C009846D70817
:1082700049070F437B0FE4001C43FF00304ED3E55A
:108280002F4EB445B4D10C0017006646CCE500274C
:108290000024E8E5002B39D00B00134300D144E75C
:1082A000C008670707438020E40800030442E1D0C8
:1082B000CB080342DED1D70849070F431C00D9E79A
:1082C000002171E700250027E9E52E002700203E68
:1082D000F740202D2FD04026751BAC405046204340
:1082E000441EA04100243843DCE6802400252403FA
:1082F000134E0027D3E5504620430700781E8741E0
:108300000024BF1860E70C0017008DE50C00170073
:108310000B4E89E51E002700203EF740202B0CD095
:108320004026F31A9C4050462043441EA041074378
:108330000024BF1848E70024D0E70024F3E7C04634
:10834000FF070000FFFF7FFF70B50E4E0D031C03FB
:1083500049005B002D0B490D240B5B0DB14204D08D
:10836000084900208B4208D070BD05430120002D34
:10837000FAD1044900208B42F6D114432000441E58
:10838000A041F1E7FF07000030B5134D0A034B0091
:10839000120B5B0DC90F0024AB4210DD0F4CA34242
:1083A0000FDC80240E4D64032243ED1A1F2D0BDDDC
:1083B0000C48C31ADA405442002900D114002000AE
:1083C00030BD094BCC18FAE7084CE840A44663449A
:1083D0009A400243EFE7C046FE0300001D04000080
:1083E0003304000013040000FFFFFF7FEDFBFFFFDD
:1083F00070B5002830D0C317C4185C40C50F2000EA
:1084000000F0C2F8174B184A1B1AD21A1F2A18DD9F
:10841000164AD21A9440002224035B05240B5B0DFC
:108420000021100024030A0D240B12052243104CD6
:108430001B05224013435B00ED075B082B4319002B
:1084400070BD210091400A000B21081AC4405B0551
:108450002403240B5B0DE3E7002500230024002206
:10846000DEE7C0461E0400003304000013040000D1
:10847000FFFF0F8010B5041E28D000F085F8154BC3
:10848000154A1B1AD21A1F2A15DD144AD21A944013
:10849000002224035B05240B5B0D00211000240344
:1084A0000A0D240B120522430D4C1B0522401343D9
:1084B0005B00590810BD210091400A000B21081AE9
:1084C000C4405B052403240B5B0DE6E70023002476
:1084D0000022E2E71E040000330400001304000041
:1084E000FFFF0F804100090E4B1C70B5DBB2460246
:1084F000750AC40F012B14DDE0239B006D07360BBA
:10850000CB1800210A0D280012051C4D32435B05D3
:108510002A405B0813435B00E4075B082343190010
:1085200070BD002914D1002D1ED0280000F02CF8B9
:108530000A281CDC0B232A001B1ADA40030015331F
:108540009D400F4B12031B1A5B05160B5B0DD8E702
:10855000002D06D0320B802636036D071643094BDB
:10856000CFE7084B0026CCE700230026C9E703002D
:108570002A000B3B9A400025E3E7C046FFFF0F802F
:1085800089030000FF0700001C2101231B049842FF
:1085900001D3000C10391B0A984201D3000A083994
:1085A0001B09984201D30009043902A2105C40184B
:1085B0007047C046040302020101010100000000EF
:1085C0000000000010B5002903D1FFF7DDFF2030C7
:1085D00002E0081CFFF7D8FF10BDC046FA020000F9
:1085E0004005000040050000400500004005000077
:1085F0004005000040050000400500004005000067
:108600004005000040050000400500004005000056
:10861000400500004005000040050000E2020000A7
:108620004005000040050000400500004005000036
:108630004005000040050000400500004005000026
:108640004005000040050000400500004005000016
:10865000400500004005000040050000F202000057
:1086600040050000400500004005000040050000F6
:1086700040050000400500004005000040050000E6
:1086800040050000400500004005000040050000D6
:10869000400500004005000040050000EA0200001F
:1086A00002030000CA020000DA020000D202000049
:1086B0000200000003000000FFFF0000FFFF0000B9
:1086C0000400000005000000060000000700000094
:1086D000FFFF0000FFFF0000FFFF0000FFFF0000A2
:1086E000FFFF0000FFFF0000FFFF0000FFFF000092
:1086F00008000000090000000A0000000B00000054
:108700009A1200009A1200009A1200009A120000B9
:108710009A1200009A1200009A1200009A120000A9
:108720009A1200009A120000B4120000B412000065
:10873000B4120000B4120000B4120000B412000021
:10874000B4120000221200003C1200005612000079
:10875000B4120000B4120000B4120000B412000001
:108760001C120000B4120000B4120000B412000089
:10877000B4120000B4120000B4120000B4120000E1
:10878000B4120000B4120000B4120000B4120000D1
:10879000B4120000B4120000B4120000B4120000C1
:1087A000B412000078120000B4120000B4120000ED
:1087B000B4120000B4120000B4120000B4120000A1
:1087C000B4120000221200003C12000056120000F9
:1087D000B4120000B4120000B4120000B412000081
:1087E0001C120000B4120000B4120000B412000009
:1087F000B4120000B4120000B4120000B412000061
:10880000B4120000B4120000B4120000B412000050
:10881000B4120000B4120000B4120000B412000040
:10882000B41200007812000053656E6420746F204B
:108830004E6F64653A20436F6D6D616E64203D201C
:10884000256420282578293B2052535349207265FE
:108850006365697665642066726F6D204E6F64652E
:10886000203D20252E3032660D0A00000D0A0D0A2B
:108870002D2D2D2D2052582066726F6D205941529A
:108880004D204E6F6465202D2D2D2D2D2D2D2D2D40
:108890002D2D2D2D2D2D2D2D2D0D000052656365B7
:1088A00069766564202564206279746573206F6E33
:1088B0002073657276696365202564206368616E44
:1088C0006E656C2025640D0A00000000446174612F
:1088D00020526563656976656420205B25645D0DC3
:1088E0000A00000052783A2000000000253032587B
:1088F0000000000020253032580D0A0048617276D1
:10890000657374312049443A203078253034582535
:1089100030345825303458253034580D0A000000C2
:108920004E756D204D657373616765205265636593
:1089300069766564203D202564202830782530380C
:1089400078290D0A000000004E6F646520566F6C98
:1089500074616765206F6E20504130333A20307863
:108960002530347820282564290D0A0052535349B4
:108970002052656365697665642066726F6D204E6E
:108980006F64653A20252E32662064426D0D0A0020
:10899000525353493A20252E32662064426D0D0A07
:1089A0000000000052784572726F723A2025640D03
:1089B0000A000000636865636B73756D2072656300
:1089C0006569766564203D203078253032580D0A7F
:1089D00000000000636865636B73756D2063616CF4
:1089E00063756C61746564203D20307825303258A1
:1089F0000D0A00002D2D2D2D2052582066726F6D0E
:108A0000205941524D204861727665737431202D92
:108A10002D2D2D2D2D2D2D2D2D2D2D2D2D2D2D2D86
:108A20002D0D00000D0A0D0A2D2D2D2D205478201E
:108A3000746F205941524D204E6F6465202D2D2DAD
:108A40002D2D2D2D2D2D2D2D2D2D2D2D2D2D2D0D76
:108A5000000000004461746120746F2053656E64EF
:108A6000205B25645D0D0A0054783A200000000068
:108A70000A0D5465737420434D332D5445535420CF
:108A80002D2056657220302E390A0D0031363A33CA
:108A9000393A303600000000466562202039203225
:108AA000303138005941524D20434D332030312070
:108AB000323031382025732025730D0A0000000064
:108AC00053656E736F722044617461205061636BF3
:108AD0006574204C656E677468203D2025640D0A1E
:108AE000000000006370756878203D2025640D0A41
:108AF0000000000053657269616C4E756D626572AD
:108B00003A203058202530782025307820253078BC
:108B1000202530780D0A00005941524D5F5365748D
:108B2000506F6C6C696E674D6F646500546F67675A
:108B30006C6520592D534441203D2025643B200085
:108B4000546F67676C6520592D53434C203D202599
:108B5000643B2000436F6E736F6C654F6E203D2049
:108B600025640D0A000000005941524D5F566572A0
:108B7000626F7365203D2025640D0A004E657720E5
:108B8000506572696F64204E6F6465205478203D93
:108B9000202564206D730D0A000000000D0A594164
:108BA000524D20434D332068656C700D000000006D
:108BB00063203D20746F67676C6520436F6E736F31
:108BC0006C654F6E0D00000079203D20746F676763
:108BD0006C65205941524D5F566572626F73650D29
:108BE00000000000312E2E30203D20506572696F4C
:108BF00064204E6F646520547820313D32733B20F1
:108C0000323D34733B202E2E20303D3230730D0028
:108C100061203D20746F67676C6520595F53444144
:108C200020616E64207265616420414443730D00CD
:108C300062203D20746F67676C6520595F53434C19
:108C400020616E64207265616420414443730D00AD
:108C500068203D207072696E7420746869732068A2
:108C6000656C70206D656E750D0A0D004144435FA3
:108C7000302025643B2000004144435F31202564BF
:108C80000D0A00000D2300000D2040005941524DF7
:108C900020496E697420446F6E652E2E2E0D0000E3
:108CA0005941524D20506F7765724F6E20446F6E60
:108CB000652E2E2E0D0000004572726F72206174B9
:108CC0002025732C204572726F72436F64653A20C1
:108CD00025640D0A00000000446F6E652025732096
:108CE0005B3078255820307825585D0D0A0000004B
:108CF0005941524D5F4C6962733A2044617461205E
:108D00005265636569766564205B33325D0D0000F2
:108D10002030782530582C20000000005941524D59
:108D20005F53657449646C654D6F646500000000B5
:108D30005265672E204745544556454E5442595476
:108D400045533A2000000000307825582C200000C0
:108D50005941524D5F53657453797374656D4D6F0E
:108D600064652054584D6F64650000005941524DB0
:108D70005F57726974655478507265616D626C6595
:108D8000000000005941524D5F5772697465547874
:108D90004669666F0000000054584C6F6F70205396
:108DA0007461727465640D0054584C6F6F70204587
:108DB0006E646564206174206379636C65203A2079
:108DC0002564205B2564206D735D0D0A00000000A2
:108DD000545820456E646564206F6E20736572760A
:108DE0006963653A202564206368616E6E656C3A3C
:108DF0002025640D0A00000000080042000C00421B
:108E00000010004200140042922C00008E2C000042
:108E10008E2C0000F02C0000F02C0000A62C00008E
:108E2000982C0000AC2C0000DE2C0000782D0000F7
:108E3000582D0000582D0000E42D00006A2D000080
:108E4000862D00005C2D0000942D0000D42D000024
:108E500060000020494E4600696E66004E414E009B
:108E60006E616E0030003031323334353637383988
:108E70004142434445460030313233343536373889
:108E80003961626364656600496E66696E6974790A
:108E9000004E614E000000000000000000000000D5
:108EA00000000000000000000000000000000000C2
:108EB00000000000000000000000000000000000B2
:108EC00000000000000000000000000000000000A2
:108ED0000000000000000000000000000000000092
:108EE0000000000000000000000000000000000082
:108EF00000000000000000000080E03779C341431B
:108F0000176E05B5B5B89346F5F93FE9034F384DEF
:108F1000321D30F94877825A3CBF737FDD4F15759B
:108F2000000000000000F03F0000000000002440AE
:108F300000000000000059400000000000408F4089
:108F4000000000000088C34000000000006AF840F4
:108F50000000000080842E4100000000D012634118
:108F60000000000084D797410000000065CDCD418E
:108F7000000000205FA00242000000E8764837426F
:108F8000000000A2941A6D42000040E59C30A2420D
:108F90000000901EC4BCD64200003426F56B0C4382
:108FA0000080E03779C3414300A0D8855734764329
:108FB00000C84E676DC1AB43003D9160E458E1438A
:108FC000408CB5781DAF154450EFE2D6E41A4B44FF
:108FD00092D54D06CFF08044F64AE1C7022DB54444
:108FE000B49DD9794378EA440500000019000000D7
:108FF0007D000000232D302B2000686C4C0065663E
:1090000067454647004300504F534958002E000023
:109010002020202020202020202828282828202028
:109020002020202020202020202020202020202040
:1090300088101010101010101010101010101010B8
:109040000404040404040404040410101010101098
:109050001041414141414101010101010101010171
:1090600001010101010101010101011010101010A5
:109070001042424242424202020202020202020242
:10908000020202020202020202020210101010206A
:1090900000000000000000000000000000000000D0
:1090A00000000000000000000000000000000000C0
:1090B00000000000000000000000000000000000B0
:1090C00000000000000000000000000000000000A0
:1090D0000000000000000000000000000000000090
:1090E0000000000000000000000000000000000080
:1090F0000000000000000000000000000000000070
:10910000000000000000000000000000000000005F
:10911000BC6400000C6400000C6400000A640000E1
:10912000AE640000AE640000A46400000A640000A5
:10913000AE640000A4640000AE6400000A64000095
:10914000B4640000B4640000B4640000446500002E
:10915000AC7100008E710000487100006670000064
:1091600048710000807100004871000066700000C6
:109170008E7100008E71000080710000667000002A
:109180005E7000005E7000005E700000C47300003E
:109190000C7A0000CC780000CC780000C878000081
:1091A000E4790000E4790000D6790000C878000076
:1091B000E4790000D6790000E4790000C878000066
:1091C000EC790000EC790000EC790000F07B000005
:1091D000F8B5C046F8BC08BC9E467047DD000000EC
:1091E000F8B5C046F8BC08BC9E467047B500000004
:0891F00020D0FF7F0100000008
:1091F800BFF35F8F01380028FAD17047FFFFFFFFE8
:10920800B80B00000CA0800040A08000E80300001C
:10921800000000000078786E7837006E6E373200F4
:1092280000000000000041550000323700464600AB
:1092380004708E0A55551055560000004050604184
:1092480051614252624353634454640160000020F8
:1092580000000000B88E0000D88E0000988E000034
:1092680000000000000000000000000000000000F6
:1092780000000000000000000000000000000000E6
:1092880000000000000000000000000000000000D6
:1092980000000000000000000000000000000000C6
:1092A80000000000000000000000000000000000B6
:1092B8004300000000000000000000000000000063
:1092C8000000000000000000000000000000000096
:1092D8004300000000000000000000000000000043
:1092E8000000000000000000000000000000000076
:1092F8004300000000000000000000000000000023
:109308000000000000000000000000000000000055
:109318004300000000000000000000000000000002
:109328000000000000000000000000000000000035
:1093380043000000000000000000000000000000E2
:109348000000000000000000000000000000000015
:1093580043000000000000000000000000000000C2
:1093680000000000000000000000000000000000F5
:1093780043000000000000000000000000000000A2
:1093880000000000000000000000000000000000D5
:10939800E95D0000995D0000000000000F900000EA
:1093A8000D900000F98F0000F98F0000F98F000080
:1093B800F98F0000F98F0000F98F0000F98F000085
:1093C800F98F0000F98F0000FFFFFFFFFFFFFFFF8D
:1093D800FFFFFFFFFFFF0000010041534349490021
:1093E8000000000000000000000000000000000075
:1093F80000000000000000000000415343494900FC
:109408000000000000000000000000000000000054
:0C94180000000000000000000000000048
:040000030000323D8A
:00000001FF
